:020000040800F2
:1050000068350020D550000815AB00086D9E0008DB
:105010000000000000000000000000000000000090
:105020000000000000000000000000008DB9000832
:10503000000000000000000091B0000869C00008F6
:10504000E7500008E7500008E7500008E750000864
:10505000E750000859680008E75000086968000830
:1050600000000000E7500008E7500008E750000883
:10507000E7500008E9A10008E7500008E7500008E1
:10508000E7500008E7500008E75000080000000063
:10509000E7500008E7500008E7500008E750000814
:1050A000E7500008E7500008E750000875CE0008F8
:1050B00085CE000829A300080000000000000000C1
:1050C0000348854600F040FD0048004751E90008CC
:1050D000683500200448804704480047FEE7FEE7A3
:1050E000FEE7FEE7FEE7FEE729C10008C150000821
:1050F00030B50B46014600202022012409E00D4670
:10510000D5409D4205D31D469540491B25469540F7
:1051100040191546521E002DF1DC30BDF0B51FB40C
:105120000646002082B005464024019100901BE015
:10513000019922460F46304600F0EAFB049A059B8F
:10514000801A994110D310461946224600F0D0FB30
:10515000361A8F410197224601200021009F00F05E
:10516000C7FB38184D4100902046641E0028DFDC44
:10517000019B00982946324607B0F0BD03460B4319
:105180009B0703D009E008C9121F08C0042AFAD2FD
:1051900003E00B780370401C491C521EF9D2704783
:1051A000D2B201E00270401C491EFBD270470022BF
:1051B000F6E710B513460A4604461946FFF7F0FF16
:1051C000204610BD30B505462A460B4610781C789F
:1051D000521C5B1C002801D0A042F7D0002C03D049
:1051E000002802D06D1CEFE7284630BD421C017834
:1051F000401C0029FBD1801A704730B504460020BE
:10520000034600E05B1C934203D2E05CCD5C401B94
:10521000F8D030BD70B5064608F0A8F90468054618
:105220000A220021304600F097FB2C6070BDF8B5D3
:1052300002464A40D40F42004B0052085B089A4293
:1052400002D20246084611464A0023D0C30D4A0046
:10525000DDB2120EAD1A202D35DA49020126490AB7
:10526000F6058A19002C00D0524220214F1B11460E
:10527000B9402A411018C20D9A4221D0002C17D0F3
:10528000012D08DCDA05801AD20F8019D207DBB2B3
:1052900000F0A2FBF8BDDA05801A012340001B06CE
:1052A000C01880185A428018CA0F1043490007E0FE
:1052B0004908C2071143DA05801A8019400880188E
:1052C00000F082FBF8BD61000122511A001BF7E7D4
:1052D0000122D2075140AAE70122D2075040A6E797
:1052E000024670B54A40D30FDB0740002DD04A007C
:1052F0002AD0010E140E000212020919400A520AA5
:105300008418E50104465443000A120A2E0450434F
:10531000A4194219200CC543AA18120C0125AD038B
:10532000521C521912047F39240400D0521C10431D
:1053300001D44000491EC2B20C06C0092018401C0E
:105340004008802A02D003E0002070BD40084000E1
:10535000002900DA0020184370BD70B502464A40AB
:10536000D50F40004A00ED0740085208002814D02D
:10537000002A12D0C40DD30D41020120C0055202F3
:10538000490A520AE41A091812187D34914201D3CD
:10539000641C00E04900002C01DA002070BD0023ED
:1053A000914201D3891A0343400849000028F7D1EC
:1053B00000290AD0914202D10121C90705E091429A
:1053C00001D2012101E00121C943E005C0184019C3
:1053D00000F0FAFA70BD420005D04200120E5242AF
:1053E0008A4201DB00207047C90508187047000099
:1053F000F0B507460846584087B0C00F04904800F3
:105400000E46590040084908BC1A884105D2384662
:1054100031461E4617460B460246580040081043C8
:105420004CD0300D039040055900400D490D0590BA
:10543000401A0290402872DA18030121000B090576
:105440000843019004980092002805D00199524227
:105450000020884100920190029840210A1A019987
:10546000009800F045FA05460C466B4607CB00F065
:1054700060FAC0197141039A0E0D0023D7175640E8
:105480001A467A40164344D0049A002A2DD0029A34
:10549000012A039A15DC1205C01A9141012636052E
:1054A000001C7141D20F059ED20700930192029613
:1054B0002A46234600F0D6FA07B0F0BD38463146FA
:1054C000FAE71605224A0F46B218C01AB741012161
:1054D0000905001C4F4100187F41114618187941F9
:1054E000E20F10436D19644113E0E2076D081543A4
:1054F0006408C2071443039A01261205C01A914199
:105500003605001C7141CE07400830434908C018D9
:1055100051412A46234600F098FACDE7FFE7049868
:1055200001224000C117121A00238B410498314612
:10553000C417381AA141EEE730B40124E4076340F0
:1055400030BC55E730B40124E407614030BC4FE77C
:105550000000E0FFF0B51FB488B00B990998002453
:1055600048400999C00F490049080991C0070B99A3
:105570000090490049080B9109990898A6460843EC
:105580001CD00B990A98084318D0099801244000B0
:10559000420D4800410D099824050003000B2043EB
:1055A00009900B980003000B20430B9050181C49E6
:1055B0004018002201901446104605E000200146E4
:1055C0000DB0F0BD032801DA034600E003239C463A
:1055D000C11A0AAE0AE05F0008ADED5B4F00F75B51
:1055E0007D430027AA187C41491C5B1E6145F2DD02
:1055F000410004AB5A522104120C0A43240C401CF3
:105600000828DFDB01980290009970460191009014
:10561000059B049A0799069800F024FAD0E7000049
:105620000DFCFFFFF0B50C465C4085B0E40FE407CD
:1056300003944C0000266408590094464908024629
:105640000296224321D062460A431ED06200570DC3
:105650004A000E032303550D012402462C4924055C
:10566000781B1B0B360B40182343264361460090E2
:105670001C46501AB44103D30098401C009002E02D
:10568000921800985B41002803DA0020014605B01B
:10569000F0BD0020012109050746864611E0644659
:1056A0001D46141BB54106D36546521BB3417446D3
:1056B00007430C43A646CD074008490828439218E3
:1056C0005B4105460D43EAD11046184313D06046AE
:1056D000194650407140084306D06046101AB34145
:1056E00006D20122002306E000220123DB0702E0AC
:1056F0000122D2435310009874460105381C6141C1
:10570000029C039D0019694100F09FF9BFE700006A
:10571000FD03000070B54B005B0803430BD04B004A
:105720005C0D002633466542B341D417AD1AA34140
:1057300002DB0020014670BD12053018514170BDDA
:1057400010B500229623114600F046F910BD000066
:105750000EB5C217C10F5040CA0740180021054BB3
:105760000293019200910A460B4600F07BF903B0C8
:1057700000BD0000330400000EB505490291002170
:1057800000910A460B46019100F06CF903B000BD90
:1057900033040000410040020122400AD205090EF4
:1057A00080187F2901DA00207047962903DC9622B1
:1057B000511AC840704796398840704770B5CD0F70
:1057C0004A0009030123090B1B0519430B4BED0785
:1057D0000024520D9A4201DA002070BD074B343389
:1057E0009A4203DC9A1A00F093F802E00449511837
:1057F00088402C43F1D0404270BD0000FF03000000
:10580000CDFBFFFF4A0009030123090B1B051943C8
:10581000094B10B5520D9A4201DA002010BD064B1B
:1058200034339A4203DC9A1A00F072F810BD03492F
:105830005118884010BD0000FF030000CDFBFFFFA2
:10584000C20FD207400040080BD0C10D0723DB0177
:10585000C91840020905400A1143C2084007114314
:10586000704700200146704710B5002904DB012471
:10587000E40740428C412146002B04DB1C460123F7
:10588000DB075242A3418B4200D1824210BD00008F
:1058900010B5002904DB0124E40740428C41214675
:1058A000002B04DB1C460123DB075242A341994233
:1058B00000D1904210BD0000CB0FDB07490010B5AE
:1058C000490802460A4307D00A0D07240903E401E8
:1058D000090B121B002A01DC002010BDC900440F77
:1058E0000C43C100E018D205801800F06DF810BD1F
:1058F00010B5202A04DB0146203A9140002010BD5B
:10590000914020239C1A0346E3401943904010BD68
:1059100010B5202A04DB0846203AD040002110BDF3
:105920000B46D340D0402024A21A91400843194688
:1059300010BD10B5202A06DBCB170846203A1041CF
:10594000C1170B4306E00B461341D0402024A21A96
:1059500091400843194610BDF7B5009C0F4600263C
:105960002578641C002D05D000F000F90068405D2A
:10597000C007F5D12B2D02D02D2D18D0641E39462D
:105980002046029A00F0F6F8002F04D03968A142B0
:1059900001D1009939607105022400290BDA4042D7
:1059A000002803DD07F0E2FD0460A007FEBD012032
:1059B00080020643E3E70028F8DA07F0D7FD046029
:1059C0000048FEBDFFFFFF7F002904DA401C4900AC
:1059D00001D140084000704770B40024050C05D187
:1059E0001024000402D1002921D01124050E01D178
:1059F00000020834050F01D10001241D850F01D1DB
:105A00008000A41C002801DB4000641C002908D091
:105A100020252E1B0D46F540A14000D00121294331
:105A2000084301061B1B000ADB1D02D5002070BCC9
:105A30007047DB05181880180029F8DA401C490067
:105A4000F5D170BC40084000704710B5002B08DA53
:105A50000024401C614192185B411A4301D1400867
:105A6000400010BDF0B51FB482B005460C0003D055
:105A7000084607F013FD02E007F010FD2030024653
:105A8000009021462846FFF733FF049B059A044601
:105A90000F4618431143084314D0184610431BD037
:105AA000009840210A1A18460599FFF731FF05466C
:105AB0000E46009A05990498FFF71AFF084305D08F
:105AC000012004E02046394607B0F0BD0020C11790
:105AD00005430E432C43374300990E986305401A43
:105AE0007905E40A00220C43FD0A0A3002D50020A1
:105AF0000146E9E70105101969410C9C0D9D00194B
:105B00006941FFF7A2FFDFE74A0009030123090B00
:105B10001B0519430A4B10B5520D9A4202DA0020B8
:105B2000014610BD064B34339A4203DC9A1AFFF744
:105B3000EFFE10BD034BD218FFF7DAFE10BD0000D8
:105B4000FF030000CDFBFFFF064C0125064E05E0DC
:105B5000E36807CC2B430C3C98471034B442F7D38E
:105B6000FFF7B2FA9CF00008BCF00008004870474C
:105B7000FCEE0008F7B582B0029C00272078641C78
:105B800015460197302802D0002D15D015E0207859
:105B90000127641C782804D0582802D0002D09D091
:105BA0000BE0002D01D0102D07D100271025207803
:105BB000641C02E0082500E00A250026009610E09B
:105BC0000099012769430818020C294680B27143E5
:105BD00000908E183804864201D30120019020786D
:105BE000641C294600F019F80028E9DA0398002817
:105BF00005D0002F01D0641E00E0029C04600198D3
:105C0000002806D007F0B2FC02210160C81E05B0D2
:105C1000F0BD009930040843F9E73A2800D2303843
:105C2000202302469A43412A01D31046373888423E
:105C300001D30020C043704770B58C180578401C14
:105C40006B075B0F01D10378401C2A1106D1027843
:105C5000401C03E006780E70401C491C5B1EF9D105
:105C60002B0705D40023521E0DD40B70491CFAE7F4
:105C70000378401CCB1A921C03E01D780D70491C60
:105C80005B1C521EF9D5A142D8D3002070BD70B55F
:105C9000044620688168490727D58168102549078F
:105CA000002905DA8168890702D481682943816067
:105CB00001F0ECFD064620688068400715D501F02C
:105CC000E5FD801B0A280CD920688068400708D5AC
:105CD000606D28436065A06D01210843A065012027
:105CE00070BD206880684007E9D4002070BD0000C6
:105CF00038B50446094808490068FFF7F9F96043D8
:105D000000900098002805D00098401E0090009850
:105D10000028F9D138BD000040420F00F4010020F6
:105D2000F8B50446206881688907890F012934D1B4
:105D30000168C90731D0816805221140102501266C
:105D4000012907D0606D28436065A06D3043A065D0
:105D50000120F8BD8168022211438160216803207F
:105D6000086001F093FD074620688068C00714D0E2
:105D700001F08CFDC01B0A280BD920688068C00781
:105D800007D0606D28436065A06D3043A065012099
:105D9000F8BD20688068C007EAD10020F8BD000087
:105DA000F8B50446206881688907890F012902D166
:105DB0000168C90733D181681A4A102611400125AC
:105DC000002907D0606D30436065A06D2843A06551
:105DD0000120F8BD8168294381600120FFF788FF19
:105DE00001F054FD074620680068C043C00716D084
:105DF00001F04CFDC01B0A280CD920680068C04384
:105E0000C00707D0606D30436065A06D2843A06572
:105E10000120F8BD20680068C043C007E8D1002019
:105E2000F8BD00001700008010B50E4801F02EFBF1
:105E300000F0CCFA05F04EFF00F010FE0A480B49C6
:105E4000C08C08600A4C0020E06000F0BFF80948F0
:105E500000F088FF00F036F9207004F0A5FA002069
:105E600010BD0000B80B0000A4070020280000208F
:105E700038000020516A0008F8B503F049FD04F02D
:105E8000FBF800F017FF04F0D1FA3D4D2878002808
:105E900001D104F02DFC04F0B1FA012801D104F085
:105EA000EFF804F0ABFA374C01280DD100F0FCFDFF
:105EB000012809D12079002806D104F00FF9002823
:105EC00002D16079002802D02878012801D105F09C
:105ED00001F9287801260025002803D104F08EFA64
:105EE000012805D005F0D6F8A57126720020F8BD6E
:105EF0002548007800283FD0A079244F002807D0FB
:105F0000012829D00228F1D1E670267120A02BE0CB
:105F10003868E168411A2248C08C814202D8207A50
:105F20000128E3D1257265701EA003F0B7FB05F0D0
:105F3000BDF8A6713868E06004F0D0F80028D5D12B
:105F40001B4928460D601B490B681B490A681B4901
:105F5000096805F059FDC9E73868E168401A3C282E
:105F6000C4D9E670267116A003F098FB05F092F8EC
:105F7000A5713868E060B9E705F08CF8A571B5E760
:105F800030000020380000200200002028000020FF
:105F900047505320535543434553530D0A000000C7
:105FA000A4070020475053204F4E0D0A0000000068
:105FB00024000020180000201C00002020000020E9
:105FC000475053204F46460D0A00000010B50120EF
:105FD00008F01CFD0A4C1328A0700AD0E01C04F045
:105FE000B7F8E078A070332806D006490020C887AB
:105FF00010BD08F043FD10BD04F07CF810BD00009A
:10600000A00100206407002010B500F003F8002074
:1060100010BD000070B50524FF222407013221467F
:10602000012005F04FF81749002007F027F816491E
:10603000022007F023F81549012007F01FF8144D3E
:10604000012292032946002004F0E2F904222946A5
:10605000012004F0DDF9012212032946022004F098
:10606000D7F910222146002000F01CFE002109482B
:1060700000F0F6F80122D2022146012000F070F86B
:10608000002070BDBC05002044060020340500201F
:10609000000400502407002010B50024084801F037
:1060A00023F9611E064801F0B7F8002803D104481F
:1060B00000F08CFF0446024801F046F9204610BD6E
:1060C000A804002070B5002400F026F80D4E054607
:1060D000B04215DB00200C4A0C4B0146FFF7D8FB01
:1060E00001D264240CE031462846FFF7F1F8084954
:1060F000FFF733F90749FFF7F3F8FFF74BFB0446C7
:10610000204670BD33335340CDCCCCCCCCCC1040EA
:106110006666663F0000C84210B500F017F86420BC
:1061200001F0B4F9FFF7B8FF00F042F8044600F0C0
:1061300003F8204610BD000010B5034801228189F4
:10614000806801F09CFB10BD6416002010B5034868
:1061500000228189806801F092FB10BD6416002046
:10616000022802D30020C0437047C3000248C15038
:1061700018188280002070476416002010B50A4C61
:10618000206B00280FD16169A06A401A3C280AD30D
:10619000FFF798FFC1B205486429017001D9642155
:1061A0000170A06A606110BD00000020380000206E
:1061B00010B5FFF7E1FA0022064BFFF733FA064A63
:1061C000064BFFF7C7F9FFF777FB0121FFF703F94C
:1061D00010BD000000FEAF406666666666660A4057
:1061E00010B50D4C00232046006861680268002944
:1061F0000BD004290BD008290BD0136402F050FDFA
:10620000206802F0BFFB002010BD5363F6E79363E4
:10621000F4E7D363F2E700004C01002010B50F4C07
:10622000206802F07FFB03CC083C02F0EFFC6168C1
:106230003C20002908D004290AD0082921680968CF
:106240000AD00864002010BD216809684863F9E796
:10625000216809688863F5E7C863F3E74C0100200B
:10626000014A03C2002070474C010020F0B5444DA4
:1062700089B00024434867000246015D5C32D15377
:10628000032909D03F49A2003F4830398850641C97
:106290000B2CEFDB09B0F0BD022101553948A600F7
:1062A000F8308059FFF754FA384A394BFFF752F962
:1062B000FFF702FB686502903248A96DCC30805927
:1062C000401AFFF759FA69672867059106902D482B
:1062D0002C49A030743180598959401AFFF74CFA83
:1062E000E967A867049003917F20C0050299FEF733
:1062F000EFFFFFF7A5FA039B049AFFF72BF9059B25
:10630000069AFFF71FF90022D243FFF703FA214A4A
:10631000214BFFF71FF91A4A204B803203C2132288
:106320001206FFF717F9E96600221D4BA866FFF772
:10633000AFFA1FD200221B4BE96EA86EFFF794FA4A
:1063400018D21948C05FFFF703FA039107460022ED
:10635000164BE96EA86EFFF7FDF83A46039BFFF770
:1063600047F8FFF72BFA074930398851E87A401C83
:10637000E8728CE7034904483039885187E7000008
:10638000A0000020880E0020FFFF0100143BB11385
:106390003BB103BEFA48CE3B1835B13D19DDB141E2
:1063A000000024C000408F40AC0F00200000594086
:1063B00010B500231A4603E0845CE3189BB2521C1C
:1063C0008A42F9D3D84380B210BD000000B587B02F
:1063D000012168464170022101700D480190C801F9
:1063E000029080000490402005906946002006F04D
:1063F00091FD07480749203801610749C1610749F4
:10640000816107494161074803F078F907B000BD91
:1064100064150020356400082964000865640008DC
:1064200073640008C40F002010B50146002006F078
:1064300031FD10BD0FB400B5FFB082B0012183ABB8
:1064400049026846829A07F013F86846FEF7CEFEC6
:1064500002466946002006F075FE7FB002B008BC17
:1064600004B0184701B501226946002006F06AFE13
:1064700008BD10B50446FEF7B9FE024621460020CD
:1064800006F060FE10BD30B4446C1C252C40012584
:10649000A540046C6560046863608368102B05D0B8
:1064A000036899600068C26030BC704703689A60F6
:1064B0000068C16030BC704708B503E068460078EA
:1064C00006F0EEFE6946002006F0E4FC0028F5D058
:1064D00008BD0000F8B50A2008F0F1F8002008F027
:1064E00009F9A64C00266670A548E0646676607CD3
:1064F0000C2801D30B2060740A212171A148A670D9
:10650000A14D00782871A14A6079127840001043AB
:10651000A27D92001043227E52011043E871E06A8E
:10652000E870020A2A72401CE062A974284614220C
:1065300097491330FEF722FE954928462C22273032
:106540006031FEF71BFE9249284616225330EC318B
:10655000FEF714FE8F480021415E002903D08E4AC9
:10656000128A511801808849027850314A76407861
:1065700088761A20687289480078A872A07F2873EC
:1065800008467E49633820310A780275497841759A
:106590006D2000227C4908F07DF920790021C0009F
:1065A0001D3008F089F906F043FF022008F0D8F802
:1065B0000026EE71A674A67301202074E673784855
:1065C00001F0B8FAA0840546A6702079FFF7D4F848
:1065D000744A754BFEF7BEFF07F004FD0022734BB3
:1065E000FEF706FFFFF70EF90006C10C481980B24E
:1065F0000121C903E084884201D3401AE0846C4839
:10660000A063E078401CE070654801F093FA608474
:10661000684E53E0624801F08DFA6084664D0AE0EE
:106620005F4801F087FA80B26084E18C884202D32F
:106630008919884206D300210F2007F0ADFF2842B8
:106640002063EDD0206B411C22D0400436D581223E
:10665000D20100210F2008F0F2F80021102007F0ED
:106660009BFF41064A48490E0022A438A16407F066
:10667000E3FF07F0A5FF2065002008F03BF80020AD
:1066800007F0F3FF4248A438417A172902D008E006
:1066900006F050FF02224949401DFEF7AEFD0028DA
:1066A00036D02A4600210F2008F0C9F82079A178B9
:1066B000401C814202D0002007F0D7FF618CE08CA3
:1066C0008142A7D380198142A4D807F077FEFFF753
:1066D000CDFD3B4B2E4A0021184660328D005559A6
:1066E000854203D228462A4D4E00AF5B491CC9B2F1
:1066F0000B29F3D3984204D0278400206073012033
:1067000020702D4A002180320F2008F098F8F8BD43
:1067100008F00BF9E165A06508F0F4F8616603463E
:106720002066A0781A4A401CC0B2A070AB3A157A15
:1067300069460D70527A4A7005464200144809882D
:106740008152134A82380090863A2846111F05F07C
:1067500081F90F4A0321903251551046A900303873
:1067600040586063A06C2628A8D1114668005C31AF
:10677000411807488C38008808809FE7A000002057
:106780003F420F0038000020A00C002054000020E1
:10679000F80D00207E000020A40700206C000020DF
:1067A000040500209A9999999999E13F00000840C1
:1067B000A0860100983A000000D027245C00002049
:1067C000FFFF01001449012048720A4602205E3290
:1067D000507203203C3A507204200E3A50720F4817
:1067E0000D4B0078087022310870203108770C4971
:1067F0005A1C087858714978997123331871597166
:10680000203318775977107551751A461E32107556
:1068100051751076517670472C0C002062000020D4
:106820005C00002010B505F089F8202005F0EEFB93
:10683000012007F0EBFD002005F0E8FB044807F01D
:1068400083FC044807F04CFF002007F081FF10BDD7
:10685000880000208380000010B5012000F042FF76
:10686000022000F03FFF10BD10B5202000F03AFFDD
:10687000802000F037FF10BD10B4084900234B61A1
:1068800007494A684C1522434A604A680824224353
:106890004A60C009C001036010BC70474C2E002044
:1068A000002002407FB500250C460646039500F007
:1068B0006BFEE009029003A901960095684600F07E
:1068C000F7FD002804D000F033FE002004B070BDB6
:1068D00000F02EFE0120F9E710B5002302E0C45CB1
:1068E000CC545B1C9342FAD310BD000010B40020BE
:1068F000204A9169CB05204904D5486902231843F1
:106900004861901593699B0505D54B690124234384
:106910004B616302184393695B0505D54B690824F5
:1069200023434B61E301184393691B0505D54B696C
:10693000042423434B616302184393699B0405D5E8
:106940004B69102423434B616302184393699B03F3
:1069500004D54C6920231C434C6118439369DB0325
:1069600005D54B69402423434B61A1020843906144
:1069700010BC7047002002404C2E002070B5044629
:1069800000F084FF0546194EB069C0070DD0601CA9
:1069900008D0002C04D000F079FF401BA04201D9A0
:1069A000032070BDB069C007F1D1B069800701D57F
:1069B0000220B061B069C00511D4B06980050ED461
:1069C000B06940050BD4B069000508D4B0698004F3
:1069D00005D4B069800302D4B069C00303D5FFF7C2
:1069E00085FF012070BD002070BD00000020024026
:1069F000F8B51746002605460C4600F0C5FD09E02F
:106A000029460220226800F0A1FD002804D1241D9F
:106A10002D1D361DBE42F3D300F08AFDBE4201D2C9
:106A20000020F8BD0120F8BD10B50849024600203D
:106A3000054B097905E044001C5B944203D0401CDF
:106A4000C0B28842F7D310BDF80D0020A00000208E
:106A500001490220887170473800002000B587B0D6
:106A6000012069464870022008700C4901914102DA
:106A700002910B4903910521490204910590694651
:106A800006F048FA8821074802F0ECFF05200122B1
:106A90001021000700F0F3FE07B000BDF41600203F
:106AA000F41A00200425002003480078002801D0B3
:106AB000002070470120704758010020F0B593B0C6
:106AC0000E460546282108A8FEF771FB03AA00928E
:106AD0002846314601AB4FA202F0F5FF0027FF43E5
:106AE00002281AD10499039802F0DDFFC2B201987E
:106AF0000178012003E0019B1B5C5940401C029B74
:106B00008342F8D8914208D1002406AB44A2314612
:106B1000284602F0D8FF0F2802D0384613B0F0BD47
:106B2000A819801E0470447049482B4602784948D1
:106B3000418804920291039405944749808809781A
:106B400001910090FF2145A201314B4803F0AEF8BE
:106B5000074680214948FEF72AFB3A4646494748FE
:106B6000FEF70CFB464D474EAF700698394600784D
:106B7000302841482AD002F0B1FD6868002846D08C
:106B800041A002F08BFD6B683A463B4900209847D4
:106B90006878002803D0FF2030606C7002E001208C
:106BA0003460687037483C4D3C4E3D4F02682B685E
:106BB0003168386804F028FF642000F067FC314831
:106BC000224604602B68316838681EE002F086FDBA
:106BD0006878002804D0FF20000230606C7002E06A
:106BE0000120346068702C4D2C4F2D482B68326882
:106BF0003968006804F008FF642000F047FC346046
:106C0000274822462B683968006804F0FDFE002002
:106C100084E700002425702A25700D0A000000007A
:106C200024252A2C252A2C252A2C252A2C252A2CD9
:106C3000252A2C25702C252A2C252A2C252A2C2582
:106C40002A2C252A2C252A2C252A2C252A2A000004
:106C50003D000020640700203800002025732C250B
:106C6000582C253032782C25782C25642C25782C2E
:106C70002564250D0A0000008C25002074160020D4
:106C8000580100201C0000204C4F52412046414634
:106C900041464146410D0A00180000202000002016
:106CA00024000020C3000248C15018188280704799
:106CB000F424002008B500206946087003E0684607
:106CC000007800F013F86946022006F0E3F8002887
:106CD000F5D008BD01490020087070475801002018
:106CE00001490120087070475801002070B51A4D05
:106CF00000262C462B78611C8034002B08D02246BD
:106D00005268022B0CD0032B09D10A2813D021E0A2
:106D1000242804D102222A7070540120606070BDC2
:106D200050546168491C61607E2913D20D28F6D148
:106D30000320287070BD50546068401C6060465449
:106D400006A1681CFEF73EFA002803D0681C6168A3
:106D5000FFF7B4FE2E7070BD042500204747412C7C
:106D60000000000001494860704700005801002001
:106D700070B53B493B4A00208300401CC0B2D15053
:106D80000C28F9D3394938480A7802754978417591
:106D900037490A780276497841763349152013310C
:106DA00048720A2007F08BFC7D20400107F0A2FC0E
:106DB0002D49002213310C2007F06CFD00210C201E
:106DC00007F07AFD06F034FB022007F0C9FC274DDE
:106DD000284C203D00210F2007F0DEFB20422863D5
:106DE000F8D0286B411C38D0400435D58122D2011F
:106DF00000210F2007F023FD0021102007F0CCFB1D
:106E000041061948490E0022C73007F015FC164C00
:106E1000C734607A15281FD102221549601DFEF77C
:106E2000ECF9002818D11148A67C2E710422611CAF
:106E30002430FEF7A3F921461331084672000C46B0
:106E40009130FEF79BF928792146420005484838E1
:106E5000FEF794F90320287070BD06F06BFB00006C
:106E6000FFFF0100580E00208D0C0020C000002004
:106E70005C00002000D02724F8B50C4605464035BC
:106E8000297C01290DD00121297401688A685207E3
:106E900009D5416D2022114341650020287401204D
:106EA000F8BD0220F8BD194B6268D8054710184E8E
:106EB0009A4215D08A6A23685B035B0B1A438A6285
:106EC0002168490305D5B1680143B1600A20FEF786
:106ED0000FFF2068800315D5B0683843B06011E01B
:106EE0008A6A23685B035B0B9A438A6221684903C1
:106EF00002D5B1688143B1602068800302D5B068D3
:106F0000B843B06000202874F8BD000001100000F4
:106F10000027014070B50446002C0AD0606D0221A4
:106F2000084360652046FEF7B2FE0546280002D001
:106F300009E0012070BD2046FEF7F2FE0546012D56
:106F400001D0012060650026012D32D02068416803
:106F50001A4A114041602168D04308602068816866
:106F600001221207914381602068C168144A1140D0
:106F7000C16020680169134A1140016120684169BC
:106F8000C908C90041612068016A0F4A11400162C5
:106F900020688030416BC909C90141632068803095
:106FA000416BC909C9014163204600F0F9F8A665A3
:106FB000666540342674284670BD000060F7FFFF08
:106FC00000023E8302FCFF3F00F000F00068006C0E
:106FD0007047000070B50446002C06D0606D264650
:106FE00000254036002802D006E0012070BDA565CE
:106FF0003574204600F0E8F8606DC00603D42068C0
:107000008168490706D5606D1021084360653574B5
:10701000012070BD616DFF220132914302221143B4
:10702000616581685C4A8907890F012902D101687D
:10703000C9072BD1032361689B07994205D05B42A6
:10704000994202D05B00994209D1016989008908FF
:107050000161206801696368194301610CE00169FD
:1070600089008908016190680F2189048843906034
:1070700090686168084390602068C168182399434C
:10708000C1602068C168A3681943C160906801218C
:107090004906884390609068A18E49060843906035
:1070A00020688168C90004D4816801221207114355
:1070B00081602068C168394A1140C1602069E26876
:1070C000022825D000200243204620300178037B8F
:1070D00049035B0019430A43216B0A43A1698903F1
:1070E0000A43E169C9030A432168CB681A43CA60AD
:1070F000616A0A46FF3AC23A05D0A26A1143226881
:10710000D3681943D16042780121012A02D00BE0F3
:107110000420D8E70078002823D0606D2022104397
:107120006065A06D0843A065E06B012820D0206851
:107130000169C90703D00169490849000161206854
:107140004169C908C900416120684169A26B1143C6
:107150004161A565606D80088000401C606500206D
:1071600070BD2068C26801231B041A43C260DBE7BC
:1071700020680269FF239B009A430261206802692C
:10718000236CA66C1A43636C33431A430261206874
:1071900002690A430261D2E7002701401902FEFF9B
:1071A00010B500680649884209D10648416B42156E
:1071B0009143416305200221000700F015FA10BD3C
:1071C000002401400010024010B586B0044614218E
:1071D0006846FDF7ECFF0E492068884216D10D483D
:1071E000416B421511434163C16A01221143C162DF
:1071F000C06A69461040059002200090032001906B
:10720000002002900520000700F078FA06B010BDBB
:107210000024014000100240F8B504460E462746FF
:107220006069403708280BD02068C068C00709D0C3
:10723000606D202108436065002038740120F8BD8E
:10724000082500E00C2500F021FB00902068006874
:10725000284219D1701C13D0002E05D000F016FB67
:107260000099401AB0420BD920680068284207D123
:10727000606D042108436065002038740320F8BD68
:10728000206800682842E5D0606D0121490208436A
:1072900060652068C16809058A0F0C21002A1BD18E
:1072A0002022125D002A17D10268120714D58268C5
:1072B00001235207002A08DB42688A434260606D5E
:1072C0001A0290431843606506E0606D2022104367
:1072D0006065A06D1843A065A069002801D12068F1
:1072E00001600020F8BD000070B504460020216850
:1072F0008968490723D425464035297C01291CD0BB
:1073000001212974E169012902D02046FEF748FDD8
:10731000002811D1616D0B4A1140FF220132114347
:1073200061650021A165297422681C211160216812
:107330008A6804231A438A6070BD022070BD02204F
:1073400070BD0000FEF1FFFF70B5044625464035D4
:10735000287C012807D001262E742046FEF797FCD2
:10736000002802D00CE0022070BD2046FEF7D8FCB9
:10737000002805D1616DFF220132914331436165DF
:107380000021297470BD30B4014620314A790023B0
:10739000022A05D00422C2630B7130BC0120704761
:1073A000026814680E25AC4314600268146864080F
:1073B00064001460446C1C22144001252A46006CB1
:1073C000A24042604D710B7130BC1846704770B5D9
:1073D0000024014620314A79022A03D00421C163E6
:1073E000012418E0026813680E25AB43136002689D
:1073F00013685B085B001360436C1C22134001257B
:107400002A469A40036C5A604D7100220A71816BC2
:10741000002900D08847204670BDF8B504468C4648
:107420000025204620300179012909D00126067166
:1074300047790021012F05D0017102252846F8BDAA
:107440000220F8BD02274771E163206801684908FE
:107450004900016061462046FFF715F8206B0028BF
:1074600005D0206801680E221143016009E0206800
:107470000168042291430160206801680A221143D7
:1074800001602068016831430160D7E770B50446A8
:1074900000F0FCF90546601C02D00448007824186E
:1074A00000F0F4F9401BA042FAD370BDE8010020BF
:1074B000F8B505460E461B4F387C012808D0012040
:1074C00038741948FFF75AFA0146080002D025E03F
:1074D0000220F8BD0020C04330606C68A868C0017D
:1074E0000019A0421AD92046FFF7C6F90E48FFF747
:1074F00045FA01460D48426808239A4342604268B3
:1075000043159A434260002901D0346006E080347C
:10751000A8686A68C0018018A042E4D800203874C6
:107520000846F8BD4C2E002050C300000020024049
:10753000054841680222114341604168012211431C
:10754000416000207047000000200240F8B50E4660
:1075500017460B4C207C012808D0012020740948D4
:10756000FFF70CFA0025002802D006E00220F8BD43
:10757000656137600348FFF701FA2574F8BD000024
:107580004C2E002050C3000012494868C0070DD09F
:10759000EFF3108072B6104ACA60104ACA6080F3D6
:1075A00010884868C00701D00120704748688007EC
:1075B0000DD5EFF3108072B6094A0A61094A0A61D3
:1075C00080F310884868800701D5012070470020AB
:1075D0007047000000200240EFCDAB890504030294
:1075E000BFAE9D8C16151413F0B50022002961D092
:1075F000012393409E460B40002B57D095082E4CFC
:10760000AD002D19AC689607360F0F27B7403C40E8
:10761000A44605242407A04201D1002419E0274CE8
:10762000A04201D1012414E0254CA04201D1022442
:107630000FE0244CA04201D103240AE0224CA042D6
:1076400001D1042405E0214CA04201D1052400E031
:107650000624B44064450FD11D4C26689E43266025
:1076600066689E436660E6689E43E660A6689E4341
:10767000A660AB68BB43AB60046855000323AB4016
:107680001C430460D408A4002418266A5507EF0E92
:107690000F25BD40AE432662C4689C43C460446865
:1076A0007546AC43446084689C438460521C0B461E
:1076B000D3409DD1F0BD0000000001400004005007
:1076C00000080050000C005000100050001C00503A
:1076D00000040140202802D10149002008607047C1
:1076E0002C00002010B504494A69024202D04861CA
:1076F000FFF7F0FF10BD000000040140F0B40022CD
:107700000B68002B6FD001270B6897403B40002B84
:107710006AD00C79A407A40F012C01D0022C10D13F
:10772000856854000326A640B543CE68A6402E4384
:1077300086604468BC430D79ED06ED0F9540254306
:1077400045600C79E443A40708D0C56854000326BB
:10775000A640B5438E68A6402E43C6600C79A407A8
:10776000A40F022C0CD1D408A40027183D6A54079A
:10777000E40E0F26A640B5430E69A6402E433E6296
:10778000056854000326A640B5430E79B607B60F28
:10779000A6402E4306604C68A403A40F50D02C4C86
:1077A000656B01263543656395082A4CAD002F199A
:1077B000BD689407240F0F26A640B543052636075B
:1077C000B04201D100261BE0234EB04201D1012678
:1077D00016E0224EB04201D1022611E0204EB04206
:1077E00003D103260CE030E02AE01E4EB04201D166
:1077F000042605E01C4EB04201D1052600E0062615
:10780000A6402E43BE60194DAC689C434E68F602FC
:1078100000D51C43AC60EC689C434E68B60200D5B2
:107820001C43EC606C689C434E68B60300D51C4357
:107830006C602C689C434E68F60300D51C432C609A
:10784000521C0B68D34000D05DE7F0BC70470000CD
:1078500000100240000001400004005000080050E9
:10786000000C005000100050001C005000040140AB
:107870000069084201D00120704700207047002AAB
:1078800001D08161704781627047000001488068C3
:1078900070470000E801002004494A6B01231A43A5
:1078A0004A6303494A6802434A6070470010024035
:1078B00000000140024881680278891881607047A1
:1078C000E801002010B50024074801684022114358
:1078D0000160032000F00AF8002801D0012401E033
:1078E00000F07CF9204610BD0020024070B504462F
:1078F0000E4D7D202978C000FDF7FAFB01460C48AB
:107900000068FDF7F5FB00F05DFF002801D00120C5
:1079100070BD042C07D200222146501E00F086F9CB
:107920006C60002070BD012070BD0000E8010020E7
:10793000F4010020704770470C480D4A816A491CC9
:107940008162C16A491CC162538F00228B4200D3FD
:107950000263084B1878012807D107480168491CC1
:107960000160022901D302601A70704700000020F4
:10797000640700203C00002058000020704770473A
:1079800070472030807B704710B50446206801683E
:10799000C943C90708D18168C943C90704D1012176
:1079A00041602046FFF7C8FF20680168C943890786
:1079B00008D48168C943890704D402214160204664
:1079C000FFF7B8FF20680168C943490708D48168F8
:1079D000C943490704D404214160204600F0FCF863
:1079E00020680168C943090708D48168C9430907A9
:1079F00004D4082141602046FFF7C0FF20680168D9
:107A0000C943C90608D48168C943C90604D41021F2
:107A100041602046FFF78FFF20680168C94389064F
:107A200008D48168C943890604D4202141602046D6
:107A3000FFF7A6FF20680168C943490608D481689A
:107A4000C943490604D4402141602046FFF797FF0F
:107A500010BD0000F8B50446002C06D0606825462D
:107A60002035A87B002802D006E00120F8BD0020C8
:107A70006873204600F046F80220A8732068844608
:107A8000C0686168012904D00122A36AD20593422B
:107A900001D11E229043184B62699A4201D0174BC4
:107AA0001840174B1840A368676A266A0B433E4389
:107AB0001E43A36A1E433043002903D12769E669A8
:107AC0003E433043012903D00121C9058B4203D134
:107AD0002369E1681943084307498A4205D0A1692F
:107AE0000A43E1690143104608436146C86001202A
:107AF000A8730020F8BD0000FFFF00003F1FFFFF3C
:107B0000FEF119FF10B50068084988420CD10848F9
:107B1000816BC20411438163002211460D2000F0E5
:107B200085F80D2000F076F810BD0000007C0040C4
:107B3000001002400068C06970470000F8B50446B4
:107B400016460222204620300546827321480268EC
:107B5000C3041A4302602068C2689B121A43C260C1
:107B60002068026901273A430261226810205060B0
:107B7000206881611021204602F0B8FB032822D042
:107B8000216808204860206846610821204602F0EC
:107B9000ADFB032819D0204602F02EFB2046FFF74C
:107BA000F0FE032813D02068816839438160206883
:107BB00001693943016120680169042211430161AF
:107BC000AF730020F8BD0320F8BD0320F8BD0320EB
:107BD000F8BD000000040140704700000448416BFC
:107BE000012211434163816B020411438163704799
:107BF00000100240002809DBC106C90E01208840A0
:107C000003490860BFF34F8FBFF36F8F70470000C9
:107C100080E100E0002805DBC106C90E0120884094
:107C2000014908607047000000E100E08207D30EC0
:107C3000FF229A408907090E9940002808DB830833
:107C400009489B001818036893430B43036070476F
:107C50000007000F0838830804489B001818C36900
:107C600093430B43C361704700E400E000ED00E084
:107C7000024801688215114301607047007000409E
:107C8000F0B4164E326875152A40154B1B6ADB0797
:107C9000DB0F002A04D0002B02D03468AC433460E0
:107CA0003468A408A400044334600E4F3C690420E7
:107CB00004433C6101290ED040BF20BF20BF396979
:107CC00081433961002A04D0002B02D03068284358
:107CD0003060F0BC704730BFF1E70000007000403A
:107CE0000000014000ED00E0F8B5044600262078D1
:107CF0005E4D80067DD55E48806BC00005D45C4833
:107D0000816B02041143816301265A480168C90549
:107D100017D40068FF210131084356490860FFF776
:107D2000B5FD074653480068C0050AD4FFF7AEFD0D
:107D3000C01B642801D90320F8BD4E480068C00567
:107D4000F4D54B4F3868032109050840626811409B
:107D5000814208D09003800F032804D13868800343
:107D600001D50120F8BD2869032109040840002835
:107D700024D00A40824221D0207880061ED528696E
:107D800088432A690121C9040A432A612A698A436E
:107D90002A612861C00511D5FFF778FD0090286998
:107DA00080050BD4FFF772FD0099411A32488142D9
:107DB00001D90320F8BD28698005F3D52078800615
:107DC00011D560688103890F032905D13A68090537
:107DD0008A43084002433A6028690322616812041A
:107DE000114008432861012E03D1B96B300781434C
:107DF000B9632078C00705D0E868A16880088000D2
:107E00000843E8602078800705D5E8680C2188439E
:107E1000E1680843E8602078400706D5E868032158
:107E20008902884321690843E8602078000706D565
:107E3000E86803210903884361690843E8602088F2
:107E4000C00506D5E968032000048143A069014309
:107E5000E9602078000606D5E86803218904884394
:107E6000E1690843E8600020F8BD000040100240CE
:107E7000001002400070004088130000F8B504466E
:107E80000D46002C1BD076480068C007C00FA842E2
:107E90001CD2734F38684008400028433860FFF711
:107EA000F5FC06463868C007C00FA8420ED0FFF7A1
:107EB000EDFC811B6B48814203D90320F8BD0120F2
:107EC000F8BD3868C007C00FA842F0D12078664FCF
:107ED000800705D5F868F0218843A1680843F86059
:107EE0002078C00772D06068022808D003280BD021
:107EF00001280ED03968890510D40120F8BD3968F1
:107F000089030BD40120F8BD3968890106D401200A
:107F1000F8BD3968490701D40120F8BDF96889081E
:107F200089000143F960FFF7B1FC0646606802284A
:107F30000FD0032820D0012831D0F8680007800F27
:107F400044D0FFF7A3FC811B464881423AD9032065
:107F5000F8BDF8680007800F022837D0FFF796FCBD
:107F6000811B4048814201D90320F8BDF868000711
:107F7000800F0228F2D129E0F8680007800F03285B
:107F800024D0FFF783FC811B3648814201D90320AE
:107F9000F8BDF8680007800F0328F2D116E0F868F2
:107FA0000007800F012811D0FFF770FC811B2D48BE
:107FB000814201D90320F8BDF8680007800F01282D
:107FC000F2D103E0F8680007800FBAD124480168B5
:107FD000C907C90FA9421CD90068214940084000BF
:107FE00028430860FFF752FC06461D480068C0079A
:107FF000C00FA8420DD0FFF749FC811B19488142F0
:1080000001D90320F8BD16480068C007C00FA84278
:10801000F1D12078400706D5F86807210902884386
:10802000E1680843F8602078000707D5F868072161
:10803000C90288432169C9000843F86000F042F88A
:10804000F9680A4A0906090F515CC84008490860E6
:1080500008480068FFF74AFC0028D3D1F8BD0000AB
:108060000020024088130000001002405AEE000871
:10807000F4010020EC010020014800687047000076
:10808000F401002000B5FFF7F7FF0449C968044A6E
:108090004905490F515CC84000BD00000010024076
:1080A00073EE000800B5FFF7E7FF0449C968044A0A
:1080B0008904490F515CC84000BD00000010024017
:1080C00073EE000870B5214EF2680C21104608408E
:1080D0001F498B0004280CD04D00082810D00C2814
:1080E00010D070680004410F491C0120C003884073
:1080F00070BD3068C00601D5084670BD184670BD19
:10810000284670BD9002134C000F205C1202940FA1
:10811000641CF268D20307D5294605F0D6F9224639
:108120000023FCF7FBFF70BD3268D20606D505F0D0
:10813000CCF922460023FCF7F1FF70BD194605F08B
:10814000C4F922460023FCF7E9FF70BD001002408D
:1081500000093D006AEE0008F0B583B00446002C2B
:108160000FD0F84EF5680C200540F7680120000498
:1081700007402078C0075BD0082D09D00C2D03D014
:108180000FE0012003B0F0BD01200004874208D1B8
:10819000306880034CD56068002849D1012003B0C5
:1081A000F0BD012061680004814203D131680143C0
:1081B000316015E0052301221B049204994206D187
:1081C00031681143316031680143316008E0316842
:1081D00081433160316801400191306890433060E3
:1081E0006068002812D0FFF751FB029030688003CE
:1081F0001ED4FFF74BFB0299401A642802D90320D2
:1082000003B0F0BD30688003F3D511E0FFF73EFB0B
:108210000290306880030BD5FFF738FB0299401AB3
:10822000642802D9032003B0F0BD30688003F3D482
:108230002078800768D5E068810604D5326820215F
:108240000A43326088430923042D17D00C2D01D135
:10825000002F13D0002842D0316899430143316088
:10826000FFF714FB0746306840072FD4FFF70EFBDB
:10827000C01B022827D9032003B0F0BD316849078D
:1082800001D500281CD071681F2212029143226977
:108290001202114371603168994301433160FFF765
:1082A00011FFF16809060A0FA749895CC840A74970
:1082B0000860A7480068FFF719FB0028DCD123E01D
:1082C000012003B0F0BD30684007CFD570681F2192
:1082D00009028843216909020843706014E030688C
:1082E000400840003060FFF7D1FA07463068400789
:1082F0000AD5FFF7CBFAC01B022802D9032003B02E
:10830000F0BD30684007F4D42078C0066BD5002D4E
:1083100015D0A069002850D03068FF2101310843F2
:108320003060FFF7B3FA07463068800536D4FFF7B0
:10833000ADFAC01B02282ED9032003B0F0BD30686F
:10834000800502D5A069002822D070680721490362
:108350008843216A084370607068217F0002000A28
:10836000090608437060206A410B491C0120C003C4
:108370008840F16809060A0F7349895CC84073494F
:10838000086073480068FFF7B1FA0028D5D12AE0E9
:10839000012003B0F0BD30688005C8D570680721A2
:1083A00049038843216A084370607068217F000296
:1083B000000A09060843706015E03168FF200130AB
:1083C00081433160FFF762FA0746306880050AD5BD
:1083D000FFF75CFAC01B022802D9032003B0F0BDEE
:1083E00030688005F4D420785A4F00072FD5606993
:1083F000002816D03869012108433861FFF746FA92
:1084000002903869800722D4FFF740FA0299401A97
:10841000022802D9032003B0F0BD38698007F3D5E4
:1084200015E03869400840003861FFF72FFA0290E4
:10843000386980070BD5FFF729FA0299401A0228FC
:1084400002D9032003B0F0BD38698007F3D4207847
:10845000400775D500200190B06BC00006D4B06B0A
:10846000012109070843B063012001903A480168DF
:10847000C90519D40068FF21013108433649086055
:10848000FFF704FA029034480068C0050CD4FFF7E7
:10849000FDF90299401A642802D9032003B0F0BD07
:1084A0002D480068C005F2D5FF20A2680130824245
:1084B00003D13969014339611BE001218902002A96
:1084C0000AD005231B029A420DD13A690A433A6148
:1084D0003969014339610CE03A6982433A6138698C
:1084E0008843386105E03A6982433A6138698843D4
:1084F0003861A068002813D0FFF7C8F902903869E6
:10850000800530D4FFF7C2F90299411A134881421D
:1085100002D9032003B0F0BD38698005F2D522E00E
:10852000FFF7B4F90290386980051CD5FFF7AEF962
:108530000299411A0948814212D9032003B0F0BDC3
:1085400019E00000001002405AEE0008F40100207B
:10855000EC01002040100240007000408813000031
:1085600038698005E2D40198012804D1B06B01215B
:1085700009078843B063606A002864D00C2D49D095
:1085800001252D0602280FD03068A8433060FFF780
:108590007DF904463068800155D5FFF777F9001B57
:1085A000022833D90320C9E73068A8433060FFF7B9
:1085B0006DF907463068800109D5FFF767F9C01BE0
:1085C000022801D90320B9E730688001F5D4E16AB7
:1085D000A06AF2680843216BFD231B049A431143F0
:1085E0000843F060306828433060FFF74FF90446D5
:1085F0003068800127D4FFF749F9001B022801D910
:1086000003209BE730688001F5D51CE030688001CD
:10861000C3D418E0012814D0F06801210904A26A2B
:10862000014091420BD10F218904E26A014091423D
:1086300005D1032189050840216B884203D0012020
:108640007CE701207AE7002078E700000248016912
:10865000022211430161704700E000E070B504465A
:10866000002C10D00220254640356874206801682F
:10867000402291430160204600F064F800206065CC
:108680006874287470BD012070BDF8B50446002CD4
:108690000ED0FF27606A0537002600280AD0266121
:1086A0006661A66225464035687C002807D00AE04E
:1086B0000120F8BD6068B842F3D0E661F1E72E749E
:1086C000204600F053F802216974206802684023B4
:1086D0009A4302602123A26860689B021A403840D6
:1086E0001043E3688A021340184323690B40217D3D
:1086F0001843C907C90F0843A169931019400843DB
:10870000E169382319400843216A8023194008434E
:10871000A16A93001940084321680860A0690421F8
:10872000000C0840616A1023194008432168486022
:108730002068C1699143C1616665012068740020A9
:10874000F8BD000010B500680649884209D1064806
:10875000416B8214914341630520E0210007FEF73D
:1087600043FF10BD003001400010024010B586B03C
:10877000044614216846FCF71AFD10492068884217
:1087800019D10F48416B821411434163C16A012220
:108790001143C162C06A002110400590E0200090A2
:1087A0000220019003200390029104910520694664
:1087B0000007FEF7A3FF06B010BD00000030014027
:1087C0000010024010B40B49401E884202D910BC70
:1087D000012070470849486108480723C26912020E
:1087E000120A4C042243C261002088610B6110BC54
:1087F00070470000FFFFFF0000E000E004ED00E034
:1088000002480169022291430161704700E000E0E3
:10881000F0B402462032137E012B22D001261676B8
:108820000223537603685D689C687027BD430F6818
:108830002F435F600068B307984208D00A4B984204
:1088400005D00A4B984202D0094B984204D18023AC
:108850009C43496821438160567600201076F0BC25
:108860007047F0BC0220704700040040000801403F
:108870000014014010B502210446203461760168DD
:108880000A6A094B1A4203D10A68520852000A6068
:1088900000F02CF80020A077A076E07620776077B3
:1088A0006076207610BD00001111000070B50546FD
:1088B000002D05D02C462034607E002802D006E032
:1088C000012070BD00202076284600F01DF802200F
:1088D0006076291D286803F02FFC0120A077A07680
:1088E000E076207760776076002070BD00680449EC
:1088F000884204D10348416B04229143416370478D
:10890000000801400010024000680449884204D178
:108910000348416B04221143416370470008014042
:1089200000100240014620314A7E012A01D0012078
:10893000704702224A760168CB6801221343CB605C
:1089400000689107884208D00B49884205D00B493E
:10895000884202D00A49884208D181684907490FF4
:10896000062906D001681143016002E00168114345
:108970000160002070470000000400400008014032
:10898000001401400168CA6852085200CA600168B8
:108990000A6A064B1A4203D10A68520852000A605A
:1089A00001212030417600207047000011110000A5
:1089B000F8B50446002625462035287E012817D024
:1089C0000120287602206876206882687727BA43DB
:1089D000FF231B029A4382600868502838D00EDCBF
:1089E000202853D006DC002850D010281ED14DE09E
:1089F0000220F8BD302849D0402817D13CE060283B
:108A000030D0702819D001221203801A0FD0904262
:108A10000CD1CB684A688968206803F0CFFB2068D6
:108A20008168012292031143816000E00126012048
:108A30006876002028763046F8BDCB684A68896899
:108A4000206803F0BBFB2068816839438160EEE752
:108A5000CA684968206803F036FC5021206803F09A
:108A6000B9FBE4E7CA684968206803F03EFC60216E
:108A7000206803F0AFFBDAE7CA684968206803F0B2
:108A800022FC4021206803F0A5FBD0E722680146C4
:108A9000104603F09FFBCAE710B586B004461421C8
:108AA0006846FCF784FB0D492068884213D10C48C6
:108AB000C26A02210A43C262C06A0191084005905D
:108AC000080300900020029003900620049069465D
:108AD0000448FEF713FE06B010BD00000008014078
:108AE0000010024000040050F8B504460D4600276F
:108AF00026462036307E01280ED001203076002A0E
:108B00000CD0042A1ED0082A33D00C2A45D00127C5
:108B1000002030763846F8BD0220F8BD294620688E
:108B200003F060FB2068816908221143816120689D
:108B3000816904229143816120688169EA68114357
:108B40008161E5E72946206803F065FB20688269BA
:108B50000121C9020A4382612068816901229202CF
:108B60009143816120688169EA6812021143816141
:108B7000CEE72946206803F06BFB2068C169082214
:108B80001143C1612068C16904229143C161206819
:108B9000C169EA681143C161BAE72946206803F058
:108BA00073FB2068C1690122D2021143C1612068B0
:108BB000C269012189028A43C2612068C169EA68E9
:108BC00012021143C161A3E770B50546002D05D01F
:108BD0002C462034607E002802D006E0012070BDC3
:108BE00000202076284600F00FF802206076291D2C
:108BF000286803F0A1FA0120A077A076E07620771C
:108C000060776076002070BD7047000070B5054643
:108C10002C462034002908D0042908D0082908D07F
:108C2000627F012A07D0012070BDA27EF9E7E27EB3
:108C3000F7E7227FF5E70220002920D0042920D081
:108C4000082920D060770122286803F0A9FA0121C1
:108C5000286889070122884208D00E49884205D039
:108C60000D49884202D00D4988420ED181684907DA
:108C7000490F06290CD001681143016008E0A07675
:108C8000E1E7E076DFE72077DDE701681143016087
:108C9000002070BD000400400008014000140140A5
:108CA00070B504460D4600222946206803F078FA84
:108CB0002068016A0B4A114203D101684908490042
:108CC000016001202034002D06D0042D06D0082D8F
:108CD00006D06077002070BDA076FBE7E076F9E76C
:108CE0002077F7E7111100007047704770B5044610
:108CF000002C1BD02420E067206801684908490047
:108D00000160206800250560206845602068856056
:108D1000204600F09BF9204680304560E5670560FD
:108D20002566656660342576002070BD012070BD23
:108D300010B504F0B9F910BDF8B504462268D06941
:108D400011689368A24D06462E40002E09D1850673
:108D500007D58D0605D5A16E002901D0204688478C
:108D6000F8BD25468035002E7FD09A4FDE07F60FDE
:108D70000F40374379D0C70706D0CF0504D5012768
:108D800017626A683A436A60820708D5DA0706D034
:108D9000276802223A626A6804273A436A604207F7
:108DA00008D5DA0706D0236804221A626A6802230B
:108DB0001A436A60020709D520220A40324305D0CF
:108DC000236808221A626B6813436B60020509D599
:108DD0004A0107D501222368D2021A626A68202359
:108DE0001A436A606A68002ABAD0800606D58806E7
:108DF00004D5A16E002901D0204688476868216803
:108E00008968490602D42821084228D0204603F068
:108E100043FC2068816849061DD5EFF310810122CB
:108E200082F31088836840229343836081F3108823
:108E3000606F00280BD068498163606FFEF7C7FA46
:108E400000288DD0606F816B8847F8BD0DE020460B
:108E5000FFF76EFFF8BD2046FFF76AFFF8BD20461A
:108E6000FFF766FF00206860F8BD266E012E7DD1F9
:108E7000C6067BD5CE0679D510231362206881689B
:108E800026464906403600294CDA626F1168496867
:108E900089B20029E8D0378B8F42E5D971831168F8
:108EA0000968890634D4EFF31081012282F3108817
:108EB00002681F01BA43026081F31088EFF310814A
:108EC000012080F310882068826852085200826076
:108ED00081F31088EFF31081012080F3108820685F
:108EE00082684027BA43826081F31088202028607E
:108EF00000202066EFF31081012080F310882068A5
:108F000002689A43026081F31088606FFEF73BFAB3
:108F100002206066308B718B401A81B22046FFF7C9
:108F2000E3FEF8BD318B728B891A89B2728B002AED
:108F3000F7D00029F5D0EFF31082012686F31088D0
:108F40000668FF272137BE43066082F31088EFF3DF
:108F50001082012080F310882068866876087600E9
:108F6000866082F310882020286000E013E0002053
:108F70002066A066EFF31082012080F3108820683D
:108F800005689D43056082F31088022060662046D4
:108F9000FFF7AAFEF8BDC50208D55B0206D5012081
:108FA000000510622046FFF7A0FEF8BD020607D5B7
:108FB0000A0605D5E16E0029F7D020468847F8BD9E
:108FC0004006FCD54806FAD5204603F095FBF8BDCF
:108FD0000F0800002001000429C5000810B5044650
:108FE000002C03D0E06F002802D007E0012010BD64
:108FF000002178200155204600F064F82420E06725
:1090000020680168490849000160204603F076FCA9
:10901000012819D0606A002802D0204603F0B6F972
:10902000206841680922D20291434160206881682A
:109030002A22914381602068016801221143016066
:10904000204603F009FA10BD012010BD10B50268DA
:109050001748184982420BD1886B01229204904331
:109060008863032189021448FEF7BEFA1D200EE032
:10907000124B052000079A420CD14A6B01239B0337
:109080009A434A6303214902FEF7AEFA1B20FEF71A
:10909000B1FD10BD0A4B9A42FBD18A6B01235B04E0
:1090A0009A438A630C21FEF79FFA1C20EFE7000029
:1090B0000048004000100240000400500038014009
:1090C00000440040F0B587B0044614216846FCF720
:1090D0006EF8314A26680025304802210323042413
:1090E000964218D1826B4E0432438263C26A0A43AD
:1090F000C262C06A6A4608400590980223C218C23C
:1091000069462748FEF7FAFA002211461D20FEF7AD
:109110008DFD1D201CE0234F0122BE421CD1456B5A
:10912000960335434563C56A1543C562C06A6D46FB
:1091300010400590032040021FC505206946000726
:10914000FEF7DCFA002211461B20FEF76FFD1B2004
:10915000FEF760FD07B0F0BD134FBE42FAD1866B3B
:1091600001277F043E438663C66A1643C662C06A0F
:109170006E46C007C00F05900C2023C6052018C6F8
:1091800069460007FEF7BAFA002211461C20FEF7D6
:109190004DFD1C20DCE700000048004000100240AC
:1091A00000040050003801400044004070B58023A6
:1091B0001B58202B01D0022070BD00290AD0002AA4
:1091C00008D0012483682403A34209D10369002B3A
:1091D00002D005E0012070BDCB0701D0012070BD99
:1091E000002303660A4C0368A3420ED05C68240285
:1091F0000BD5EFF31084012585F310881D68012637
:10920000B60635431D6084F3108803F0B1FC70BDD1
:109210000048004070B580231B58202B01D002204D
:1092200070BD00290AD0002A08D0012483682403D5
:10923000A34209D10369002B02D005E0012070BDD3
:10924000CB0701D0012070BD002303660A4C0368E0
:10925000A3420ED05C6824020BD5EFF310840125E5
:1092600085F310881D680126B60635431D6084F31A
:10927000108803F0D5FC70BD0048004010B503F025
:1092800035FF10BD7047FFB583B004460F46154645
:10929000E06F202802D0022007B0F0BD002F0AD0D6
:1092A000002D08D00120A168000381420BD1206964
:1092B000002803D007E0012007B0F0BDF80702D076
:1092C000012007B0F0BD0021842001512120E0677A
:1092D000FEF7DCFA02902646403635827582012080
:1092E000A1680003814202D12069002813D03D46C5
:1092F0000027708A00281CD0069800900022802148
:109300002046029B03F05CFD002806D02020E06789
:10931000032007B0F0BD0025EBE7002D18D0216831
:10932000287888626D1C708A401E7082708A0028BE
:10933000E2D106980090002240212046029B03F0D3
:109340003FFD00280BD02020E067032007B0F0BDD0
:1093500038882168C005C00D8862BF1CE3E7202063
:10936000E067002007B0F0BD70B50446E06F20282C
:1093700001D0022070BD00290AD0002A08D00123A4
:10938000A0681B03984209D12069002802D005E09B
:10939000012070BDC80701D0012070BDE1642046E6
:1093A0004030028242820021403005464160212047
:1093B000E067206F00281AD0154BC362236F154851
:1093C0001863236F14485863206F81632068134625
:1093D0002830266F02463046E16CFEF71EF8002862
:1093E00005D0102068602020E067012070BD216852
:1093F00040200862EFF31081012080F3108820687C
:10940000826880231A43826081F31088002070BD37
:1094100043C600088FC600083DC5000830B4C36FBE
:10942000202B02D030BC0220704700290AD0002A2D
:1094300008D0012483682403A3420BD10569002DC1
:1094400003D007E030BC01207047CD0702D030BC0C
:1094500001207047C164014640310A824A820021DE
:10946000C166842211502121C167A34202D1016942
:10947000002910D00949C166EFF31081012282F35F
:1094800010880068026880231A43026081F3108804
:1094900030BC002070470249C166EDE763CD00088B
:1094A00001CD000810B503F0B9FE10BD70470000F3
:1094B0000020014908707047A004002001200149E4
:1094C00008707047A004002070B504460D46204681
:1094D00000F02CF8012801D1801E70BD2268501CBC
:1094E000E168FBF705FE2160236921685943A36801
:1094F000C81829462269FBF741FE0020EDE710B5A8
:109500008160C2600361012444600024046010BDD6
:1095100010B504462268501CE168FBF7E9FD60685D
:10952000814201D1012010BD0020FCE710B50446A6
:109530002268901CE168FBF7DBFD6068814201D185
:10954000012010BD0020FCE770B504460D46204602
:10955000FFF7DEFF012801D1801E70BD236960681E
:109560005843A368C11828462269FBF707FE6268C2
:10957000501CE168FBF7BCFD61600020EDE770B5B1
:1095800004460D46002C01D1401E70BD00BF20686E
:10959000A842FCD32068401B206062685019E16833
:1095A000FBF7A6FD61600020EFE770B504460D46AD
:1095B000002C01D1401E70BD20684019206000BF02
:1095C000E16820688842FBD8A2685019E168FBF77F
:1095D0008FFDA1600020EEE7FFB581B004460D4687
:1095E00016460027002E06D00498002803D0E16814
:1095F0002068884203D30020C04305B0F0BD216835
:10960000E068401AA84202D20020C043F5E7A068F3
:109610004019E16888420BD9A168E068471A2168BF
:10962000E068401AE919884202D20020C043E4E70A
:10963000A268D019E168FBF75BFD316079190498E5
:1096400001600020D9E701464868704701468868F4
:1096500070470246002A01D1401E7047002050602A
:1096600090601060D16000BFF7E70146002901D18A
:10967000012070470868002801D10120F9E7002087
:10968000F7E70146002901D1012070470A68C86840
:10969000904201D10120F8E70020F6E70FB400B5B1
:1096A0000D48FFB0007882B0012805D000207FB0BF
:1096B00002B008BC04B01847012183AB49026846D8
:1096C000829A03F0D5FE6846FBF790FD0246694694
:1096D000002003F037FDEAE75401002010B5064AE8
:1096E0001278012A01D0002010BD0A460146002050
:1096F00003F028FD10BD0000540100200349096853
:109700000160022181710149086070471002002048
:1097100000BFEFF30580002800D0704707480068BD
:10972000002804D1012080F3108800BF00BF034847
:109730000068401C0149086000BFEEE7F801002006
:1097400070B504460D4600F04FF800280FD000F029
:109750004BF80B21C90140180069002807D000F020
:1097600043F80B22D2018018016902A0884700202B
:1097700070BD00001B5B481B5B4A000070B50246D1
:109780000C4600210023002A01D0002C02D1002029
:10979000C04370BD0021002316E0C8000D4D2858BD
:1097A000002810D1D8001058CD000A4E7051D800B2
:1097B00080184068CD00AD19686007480068401CFB
:1097C000054D28605B1C491C502901D2A342E4D3FB
:1097D0000020DEE71C02002018020020014800687B
:1097E0007047000018020020014800687047000020
:1097F00014020020F8B506460F46002536E0002486
:1098000018E0FFF7F1FF002813D0FFF7EDFF0B2161
:10981000C9014018006900280BD0FFF7E5FF0B23B2
:10982000DB01C01802692819C000134B195813A096
:109830009047641C052C04DAFFF7D0FF29198842F1
:10984000DFD8FFF7D1FF00280FD0FFF7CDFF0B21A6
:10985000C90140180069002807D0FFF7C5FF0B2297
:10986000D2018018016907A088476D1DFFF7B6FF78
:10987000A842C4D80020F8BD1C020020252D313696
:10988000730000000D0A00000146202902D30020C9
:10989000C0437047012218204843044B1A5000224D
:1098A00018204843C01882600020F2E7642E002090
:1098B00070B505460024002D01D1401E70BD002466
:1098C0000CE0182060430C490858002805D10121FC
:1098D00018206043084A115002E0641C202CF0D389
:1098E00000BF202C05D105A0FFF7D8FE0020C04303
:1098F000E4E72C600020E1E7642E002074696D65C8
:10990000722049442069732066756C6C0D0A000052
:1099100010B5002400BF41E01820604321490858D9
:1099200002283AD118206043401880681E4909680F
:10993000091A182060431B4A8018C06881422CD93C
:1099400018206043114640184069002820D0182094
:10995000604340180079002804D101211820604399
:1099600011500AE00221182060430E4A11500E489F
:109970000168182060438018816018226243094BF7
:10998000D218106918226243D2185169884704E03E
:10999000012118206043034A1150641C202CBBD3C2
:1099A00010BD0000642E002000020020F0B5044627
:1099B000059D202C02D30020C043F0BD02261820B4
:1099C00060430E4F3E50182060433E46801901719F
:1099D0000B48066818206043C01986601820604351
:1099E0003E468019C26018206043801943611820E8
:1099F0006043801905610020DFE70000642E00202D
:109A00000002002007480068401C0649086006481C
:109A1000026840680021521C484103490A604860BE
:109A200070470000000200200802002000BFEFF392
:109A30000580002800D0704709480068002804D03D
:109A400007480068401E064908600548006800286D
:109A500004D100BF80F3108800BF00BF00BFEAE759
:109A6000F801002070B504460D4629462046FBF754
:109A70009EFB70BD0146302904DB392902DC084613
:109A800030380EE0412904DB462902DC084637382D
:109A900007E0612904DB662902DC0846573800E04C
:109AA0000020C0B2704710B502460B46002406E005
:109AB0001078FFF7DFFF21014418521C5B1E002BBA
:109AC000F6D1204610BD0FB4F0B585B00446002095
:109AD000049000222020039000200290002C02D04D
:109AE0000C98002805D1002005B0F0BC08BC04B0DB
:109AF00018470DA80490CFE0002908D10C980078F1
:109B0000252803D10C984078652800D0C9E00C982E
:109B1000007825286ED10C98401C0C900C98007889
:109B200003900C98401C0C900398652877D004DCB7
:109B30002A2807D0642873D113E0702872D07828BF
:109B4000F9D13EE008E020780C9B1B78984202D0C7
:109B5000641C491E00E001E00029F4D100BF521C42
:109B600088E0002601960096002300252020049E10
:109B700020CE049618E02078009E002E05D12D28D6
:109B800003D10126019600960CE0302809DB392824
:109B900007DC012600960A265E430746303FF3198C
:109BA00000E003E0641C491E0029E4D100BF019ECF
:109BB000012E01D1DE43731C002D00D02B60521CFE
:109BC00058E000230025049E20CE04961FE0207854
:109BD000302806DB392804DC1E010746303FF31924
:109BE00013E0612807DB662805DC1F010646573EA7
:109BF000BB190AE043E0412806DB462804DC1F01CC
:109C00000646373EBB1900E003E0641C491E0029EC
:109C1000DDD100BF002D00D02B60521C2AE01BE0DC
:109C200024E0FFE7049E01CE04960025002325468C
:109C300009E026780C9F3F78BE4201D05B1C00E013
:109C400003E0641C491E0029F3D100BF002801D0A5
:109C500005604360521C0DE0049B01CB0493002877
:109C600000D00460521C0123029303E00120029003
:109C7000002200BF00BF029801280DD111E020781A
:109C80000C9B1B78984205D1641C0C98401C0C90CE
:109C9000491E01E0002204E00C980078002800D062
:109CA0002AE700BF0020049010461DE70FB4F8B566
:109CB00006460C46002509A8009021463046009B28
:109CC000089A03F0D5FB054600200090A54200D37A
:109CD000651E2846F8BC08BC04B01847FEB504460B
:109CE0000F4615460026002001900090002C01D060
:109CF000002D01D10020FEBD2846FBF777FA009029
:109D00000098874201D20020F5E70098381A0190A8
:109D1000002609E0A0192946009AFBF76EFA0028F0
:109D200001D1A019E7E7761C01988642F2D3002002
:109D3000E1E770B504460D46002C01D0002D02D19C
:109D40000020C04370BD012120461030FFF717FCF2
:109D500020462030A968FFF712FC0020F2E770B51A
:109D600004460D46002C01D0002D02D10020C04336
:109D700070BD012120461030FFF717FC204620302F
:109D8000A968FFF712FC0020F2E710B50446002C8A
:109D900000D110BD20461030FFF767FC012801D12B
:109DA0000020F6E720462030FFF75FFC012801D1B4
:109DB0000020EEE720461030FFF745FC0C21484319
:109DC00021684018E5E77CB504460E4600250020D2
:109DD00001900090002C00D17CBD20461030FFF790
:109DE00050FC002801D00020F6E76B4601AA31465E
:109DF00020462030FFF7F0FB002801D00020EBE7E1
:109E000020461030FFF722FC0C21484321684518FA
:109E1000A0680199401828606E600098A8602846E4
:109E2000DAE7FFB581B004460E461D4600270C2038
:109E300068430399884202D3781E05B0F0BD0C2018
:109E40002F4647432660676060688019A0600398CA
:109E5000C11BE160294620461030FFF7FAFB20467F
:109E60002030E168FFF7F5FB0020E6E7FEE70000A1
:109E700010B50E4C002208212046FDF700FD0022FF
:109E800010212046FDF7FBFC0A2004F016F9012200
:109E900008212046FDF7F3FC0A2004F00EF9002209
:109EA00008212046FDF7EBFC10BD00000004005027
:109EB00010B50E4C002208212046FDF7E0FC0122DF
:109EC00010212046FDF7DBFC0A2004F0F6F8012201
:109ED00008212046FDF7D3FC0A2004F0EEF800220A
:109EE00008212046FDF7CBFC10BD00000004005007
:109EF000F8B50024144E07462546002208213046B6
:109F0000FDF7BDFC0A2004F0D8F8012208213046F4
:109F1000FDF7B5FC6006040E10213046FDF7A8FCE5
:109F2000002801D0641CE4B2052004F0C6F86D1CC2
:109F3000EDB2082DE1D3002F03D0FFF799FF2046A3
:109F4000F8BDFFF7B5FFFAE70004005070B5154EF5
:109F50000546002208213046FDF791FC0024E8095F
:109F600001D0012200E0002210213046FDF787FCDD
:109F70006806050E0A2004F0A0F8012208213046E8
:109F8000FDF77DFC0A2004F098F8002208213046F5
:109F9000FDF775FC0A2004F090F8641CE4B2082C6C
:109FA000DDD370BD0004005010B50C4C012210210F
:109FB0002046FDF764FC012208212046FDF75FFCE6
:109FC000002210212046FDF75AFC0A2004F075F803
:109FD000002208212046FDF752FC10BD000400506D
:109FE00010B50E4C002208212046FDF748FC002247
:109FF00010212046FDF743FC0A2004F05EF8012200
:10A0000008212046FDF73BFC012210212046FDF7E8
:10A0100036FC0A2004F051F810BD00000004005086
:10A0200070B5144D0024012210212846FDF727FCAD
:10A03000062004F042F8012208212846FDF71FFC03
:10A04000062004F03AF807E0641CE4B2FA2C03D9C5
:10A05000FFF7C6FF012070BD10212846FDF708FC60
:10A060000028F1D1002208212846FDF708FC002035
:10A0700070BD00000004005010B5FCF71DFA10BDC3
:10A0800070B500F02BF8104C012816D1A0780028EC
:10A0900013D10120A07020780C490D4B0D4A0E4DB4
:10A0A0005A2802D3FF20000401E0FF2000020860CC
:10A0B0001B681268296801F0A7FC00F00FF800285F
:10A0C00000D1A07070BD00003800002024000020E6
:10A0D000180000201C0000202000002010B50448BB
:10A0E00081880068FDF7C4FB012800D0002010BD66
:10A0F0004C00002010B53721202000F070F803211B
:10A10000212000F06CF84021222000F068F808219E
:10A11000232000F064F8AA21302000F060F80A48FB
:10A1200002210187322000F05AF80121332000F08B
:10A1300056F85F21202000F052F8044800F008F89B
:10A140000A2003F0BAFF10BD64070020A30100201D
:10A1500010B501460F2000F021F8002800D00120A2
:10A1600010BD10B50446FFF71FFF3220FFF7EEFECB
:10A17000FFF756FFE0B2FFF7E9FEFFF751FFFFF7E9
:10A1800013FF3320FFF7E2FEFFF74AFF0020FFF73F
:10A19000AFFE0446FFF724FF204610BD10B50C4665
:10A1A000FFF7DFFF2070012010BD70B50D4604469B
:10A1B000FFF7FAFE3220FFF7C9FEFFF731FFE0B2EA
:10A1C000FFF7C4FEFFF72CFF2846FFF7BFFEFFF79F
:10A1D00027FFFFF705FF0A2003F06FFF70BD10B5E2
:10A1E000FFF7E3FF012010BD10B50248FDF7CCFBDF
:10A1F00010BD000004050020F0B583B00446002621
:10A20000EFF310800090012080F31088344B206819
:10A21000C21804D13349CE68032189040E408168F5
:10A220000291C168019141698569002A07D12E48D0
:10A23000826AC7043A438262826ABA4382620846EB
:10A2400028433CD026482268C24205D12548C3682D
:10A25000032292049343C36027462037002910D07D
:10A260002068026901231A430261206841610821C4
:10A27000204600F03BF8032800D1B873216808207D
:10A280004860002D10D0206801690122114301614E
:10A29000206885611021204600F028F8032800D1AD
:10A2A000B8732168102048600D482168C14206D16A
:10A2B0000C48C1680322920491433143C160206875
:10A2C0000169490849000161216802988860216894
:10A2D0000198C860009880F3108803B0F0BD0000BA
:10A2E0000084FFBF401002400010024070B50646D7
:10A2F0000D4600240B480A490068FAF7F9FE7D2153
:10A30000C90048433268401E002800D10324136866
:10A310002946994301D00028F5D1204670BD0000A0
:10A32000204E0000F401002010B50248FEF704FDA5
:10A3300010BD00003405002010B5032000F002F825
:10A3400010BD000070B5164D00262C460C3C0028B0
:10A3500011D021468978032814D001280AD1491C3C
:10A36000C8B2A0700C2817D204280FD0800028583B
:10A3700000F072F970BD00F01FFA0520FDF786F8B5
:10A38000A67001E00029F5D12868F1E705492869A0
:10A39000096800F061F970BD00F004FA70BD0000BA
:10A3A0006C0100205C00002000B587B001206946E8
:10A3B0004870022008700E490191410202910D4936
:10A3C00003918021049105906946012002F0A2FDCD
:10A3D0000948FFF76DFA00F0EFF900F02DF964205D
:10A3E000FDF754F80020FFF7ADFF002007B000BDD7
:10A3F000B4270020B42B002064010020034880789B
:10A400000C2801D000207047012070476001002017
:10A41000032802D30020C0437047C3000248C15044
:10A4200018188280002070479C270020FEB5002568
:10A43000684605710581FF270580414C0137414E73
:10A4400037E06846007900F0ABF86846027930786A
:10A450002254401C3070207855282AD16078AA28D0
:10A4600027D1607A552824D1A07AAA2821D1606802
:10A4700002903549684600890968884219D1A07957
:10A48000012811D1E079012813D1207A002810D1B8
:10A490002E4805702E4805702EA0FFF7FFF83946AC
:10A4A0002748FAF784FE3570A079022815D00328D2
:10A4B00029D001A9012002F0EDFC0028C1D0FFF74E
:10A4C0009DFF012808D1F078002805D039461C48A6
:10A4D000FAF76DFEF5703570FEBD19496846CA7908
:10A4E0000270097A41700188E120C000814201D8E0
:10A4F00069460880684604881A48C48404F0DCFB76
:10A50000214619A014E00E496846CA790270097AFA
:10A51000417000880A2802D80A20694608806846E7
:10A52000048810484038448704F0C6FB214615A033
:10A53000FFF7B4F8642003F0B9FD03F009F8000058
:10A540009C260020600100205C0000203B000020D1
:10A550003C000020CAD5B5BD475053B5C44F4B0D84
:10A560000A000000A4070020CAD5B5BDD0DEB8C4DB
:10A57000475053BFAAB9D8CAB1BCE43A25640D0A02
:10A5800000000000CAD5B5BDD0DEB8C4BEB2D6B991
:10A59000D0DDC3DFCAB1BCE43A25640D0A00000077
:10A5A00070B51E491E4B4A78012A05D18A687F2A58
:10A5B00002D29854521C8A6000220A2802D00D2828
:10A5C00004D029E001208A60487025E04A708C6838
:10A5D000002C21D018192038C277114D4868FFF798
:10A5E00053F910A221462846FFF778FB002805D032
:10A5F00029460DA0FFF752F801200BE00CA22146DE
:10A600002846FFF76BFB002806D0294606A0FFF777
:10A6100045F80220FFF796FE002070BD6001002083
:10A62000342C00206F6B00005B525D2025730A0004
:10A630006572726F7200000010B5034801228188B4
:10A640000068FDF71CF910BD9C27002010B5002004
:10A65000FFF778FE10BD00000FB430B591B015AB18
:10A66000402101A8149A02F003FF002501A8FAF77F
:10A67000BDFD024601A9012002F064FD04460A481E
:10A680007D220095074B120100214068FFF78EF9EB
:10A6900001A906A0FFF702F8204611B030BC08BCA3
:10A6A00004B0184739A30008600100205B535D2007
:10A6B00025730A0070B505460C480C4680780C28B6
:10A6C00002D00020C04370BD00F076F80520FCF7F2
:10A6D000DDFE22462946012002F034FD0520FCF76C
:10A6E000D5FE00F05FF8002070BD00006001002082
:10A6F000F8B51F4E1F4C30682169401A0A2836D918
:10A70000E078002833D0012020711B4801781B48D5
:10A71000FFF7D0FFFF2101311948FAF748FD19482A
:10A720000025057030682061E079FF21401CE07150
:10A730001548174E01601548164F0368326838688F
:10A7400001F062F96420FCF7A1FE0F48294605607C
:10A750000E4832680368386801F056F9E079042839
:10A7600002D92571E570E5710BA0FEF797FFF8BDE2
:10A7700028000020380000205A0100207416002014
:10A780009C260020600100202000002018000020EE
:10A790001C000020240000206C6F7261206275662E
:10A7A000610D0A0010B50348002281898068FDF719
:10A7B00066F810BD9C27002010B50348012281894E
:10A7C0008068FDF75CF810BD9C2700201CB50021B7
:10A7D00018480091164A01910260C1631205426057
:10A7E000816007228263012202610246C160203239
:10A7F0001170FF235170C233436281621173016390
:10A800008161042241634261C161FCF7E3FB0028DE
:10A8100001D072B6FEE708480090801301906946A7
:10A820000448FCF729FB002801D072B6FEE71CBDE6
:10A8300000240140A804002002000004F0B587B005
:10A8400014216846FAF7B3FC4148C26A04210A435E
:10A85000C262C26A0A400592C16A01252943C162E7
:10A86000C16A29400591C26A02210A43C262C06AD4
:10A87000052708403F070590002236493846FCF777
:10A88000FEFF002234493548FCF7F9FF012211038D
:10A890003846FCF7F4FF012240213048FCF7EFFF77
:10A8A0001126360400246946384601960095029424
:10A8B000FCF724FF2A48009002946946019503940E
:10A8C0003846FCF71BFF244802941838009069466C
:10A8D000019503942148FCF711FFA22000906946DE
:10A8E000019602941D48FCF709FF0920000300901F
:10A8F0000194694602941948FCF700FF1820009063
:10A90000112001900294694603941448FCF7F6FE66
:10A9100040200090032003900195029469460F485F
:10A92000FCF7ECFE2802FCF7B7FF002211460520D9
:10A93000FDF77CF90520FDF76DF90022114607208F
:10A94000FDF774F90720FDF765F907B0F0BD0000C9
:10A9500000100240108900001D410000000400505A
:10A960001099000010B5FFF731FF00F009F800F072
:10A9700099F800F0B3F800F01FF800F043F810BDAC
:10A9800010B50C480A490160E121490241600021EB
:10A990008160C160016181610C220162426141629A
:10A9A000FEF71CFB002801D072B6FEE710BD0000C8
:10A9B000004800403405002010B5114C0F482060BD
:10A9C000FF20053060600020A060E06020616061D1
:10A9D000E0610121206249026062A161A06207205A
:10A9E000E0622046FDF751FE002801D072B6FEE776
:10A9F0002068016840221143016010BD0030014011
:10AA0000CC06002010B58AB0002404940594069466
:10AA100007940894224809940094019402941F49D1
:10AA2000039401601F21846041600461F921446145
:10AA3000C160FDF73BFF002801D072B6FEE70120A0
:10AA40000003049004A91648FDF7B2FF002801D0C6
:10AA500072B6FEE71248FEF7B7F8002801D072B6CA
:10AA6000FEE7089408A90E480994FDF7D1FE0028D6
:10AA700001D072B6FEE7602000900194029400229B
:10AA8000694603940648FEF72FF8002801D072B6F5
:10AA9000FEE70348FEF700F80AB010BD00080140C9
:10AAA0002407002010B50C480A490160E121490241
:10AAB000416000218160C16001618161C1610C223E
:10AAC000016242614162FEF789FA002801D072B644
:10AAD000FEE710BD00380140BC05002010B50C4851
:10AAE0000A4901604B21C901416000218160C160B8
:10AAF00001618161C1610C22016242614162FEF724
:10AB00006DFA002801D072B6FEE710BD0044004087
:10AB100044060020FEE70000F0B58BB00A2003F0E9
:10AB2000CEFD7D20400103F0E5FDFF4C0025657062
:10AB3000FE48E064607C0C2801D30B20607420790F
:10AB40000A2801D90A202071A570207D012700283C
:10AB500003D0032801D0277600E02576F448F54E8F
:10AB600000783071F4480078F071E06AF070010A02
:10AB70003172401CE0622079B07442003046EF49E7
:10AB80001330FAF7FBFA2079EC4982004000801973
:10AB900060311330121DFAF7F1FA207906214200D4
:10ABA0004843E6498019EC311730921CFAF7E6FA6F
:10ABB000E3490020085E002803D0E24A128A1018F8
:10ABC00008802079DB4EC30098190A7842764978CC
:10ABD000817616207072B572A07F3073D2493046EC
:10ABE000203113380A7802754978417518461D30AE
:10ABF0000022314603F04EFE20790021C0001D30B6
:10AC000003F05AFE02F014FC022003F0A9FDF571D6
:10AC1000A574A57301202074E573CB48FCF78AFF67
:10AC2000A0840646A5702079FAF7A6FDC74AC84B4E
:10AC3000FAF790FC03F0D6F90022C64BFAF7D8FBDE
:10AC4000FAF7E0FD0006C00C801980B20121C903AB
:10AC5000E084884201D3401AE084BF48A063E078D2
:10AC6000401CE070B848FCF765FFB44E6084A43E19
:10AC7000304622300890001F0290001F0190801E75
:10AC8000079036E1B048FCF755FF6084B34F0BE006
:10AC9000AD48FCF74FFF80B26084E18C884203D35B
:10ACA000AF4A8918884206D300210F2003F074FCB4
:10ACB00038422063ECD0206B411C21D040047DD56C
:10ACC0008122D20100210F2003F0B9FD00211020C4
:10ACD00003F062FC41069948490E27460022A43839
:10ACE000A16403F0A9FC03F06BFC3865002003F0BD
:10ACF00001FD002003F0B9FC717A1729C1D101E0F0
:10AD000002F018FC02229749701DFAF776FA002823
:10AD1000B7D103F00AFEF965B86503F0F3FD796673
:10AD20003866B8786946401CB8708448AB38027AF7
:10AD30000A70407A487008880990398C88427ED120
:10AD40007E4903209031087008980090236E0020FF
:10AD5000029A019900F07EFE7648834F8C30C08EB7
:10AD6000388074488C30008FA0837748FCF7E2FE6F
:10AD7000608403F023FBF07C0009607513D002228D
:10AD80007849701DFAF739FA00280CD10120694979
:10AD9000A074C871A06CCA311638C2B26748E27498
:10ADA0009C30FAF7EBF97148057064486030006830
:10ADB0006063A063E063F17C090700E08CE0090FA9
:10ADC000032900D02175A16C262917D15949564A6B
:10ADD0008C31C98F1185594B079AB43312881A8761
:10ADE00088420ADD002808DD002906D0E07D411CEC
:10ADF000E175052802D9257000E0E575E5700120B0
:10AE0000A073E073A08B5A49FF30C33080B2A08397
:10AE100088420BD949424018A08338887D21401CC4
:10AE200080B2C9003880884200D33D8038887D21B7
:10AE3000C9004843A18B4018206468E0FFE7FBF796
:10AE4000F3FD04900898009004983B6E401CC0B23B
:10AE5000029A019900F0FEFD3849049890310322CE
:10AE600008184270049830398000844640184068C1
:10AE70007863B86C262806D104988C3140004118BC
:10AE80000798008848802D482A4930308C3160442A
:10AE9000898F0180274861460B180022796E386E31
:10AEA0003C46163398540F06000A3843090A521CD0
:10AEB000042AF7DBE16C606B88421ADA1F496346AB
:10AEC0003031C958002914D0012901D0814210DD48
:10AED000E064099806900CE03A4600210F2003F048
:10AEE000AEFC2079A178401C814202D0002003F002
:10AEF000BCFB608CE18C884200D2C3E6184A8918FA
:10AF00008842FAD8A07B012801D00221A17303F066
:10AF100055FA124A00210F2003F091FCE078002836
:10AF20003BD00A282AD925E0A00000203F420F008C
:10AF300038000020A00C00203D000020F80D00206B
:10AF40007E000020A4070020040500209A9999990A
:10AF50009999E13F00000840A086010000D0272415
:10AF6000983A00005C00002060000020540000209F
:10AF7000E7030000E5702570FBF7ACFAFBF776F904
:10AF8000A07C002857D03C4E3178617270782072D6
:10AF9000B278E271022917D04DE0A06BE16C323833
:10AFA00081420FDAA1792046491CC9B2A171022958
:10AFB000E4D9857106990184022101702573FBF79C
:10AFC000D7FEDBE7A571D9E710280ED02B4F062856
:10AFD00015D0C8282FD23818F11CFAF7CFF803F093
:10AFE0006BFE642003F062F88AE6254F3868400063
:10AFF000000E20D1F078FAF7A3FB38601BE00222A4
:10B00000F11CB81DFAF7F9F8002814D0207AE2797B
:10B010003818F11CFAF7B2F803F04EFE7D20F988DB
:10B02000C000FAF765F8174908800146C820FAF70A
:10B030005FF815490880104F00269C3F12E00E492A
:10B0400075008439785B495B884209D00220207002
:10B05000FBF78EFE0020207307490120B4394853C6
:10B06000761CF6B220798642E9D3084A00210F20E7
:10B0700003F0E5FB0BB0F0BD940E00206407002048
:10B08000700000206C0000207800002080D0272471
:10B090007047000010B50448002281898068FCF7E1
:10B0A000EEFBFBF717FE10BD8C26002010B5044800
:10B0B000012281898068FCF7E2FBFBF711FE10BDDD
:10B0C0008C260020C3000248C150181882807047A7
:10B0D0008C260020F0B585B04848FBF71BFF484898
:10B0E000FDF7BCFA4748FDF7C5FB4748FDF7FEFDF5
:10B0F0004648FDF7FBFD4648FDF7F8FD00F0A0FCD3
:10B1000014216846FAF753F8002410261127052069
:10B11000029469460007019700960394FCF7EEFA43
:10B12000F5010520029469460007019700950394F4
:10B13000FCF7E4FAFDF764FB3648816B0204114327
:10B1400081633548016804221143016001210846EA
:10B15000FCF796FDFDF77AFA00F08CFFFFF702FC92
:10B16000002001F051FF012001F04EFF022001F00C
:10B170004BFF0096012605200294694600070196C0
:10B180000394FCF7BBFA0520012210210007FCF70D
:10B1900076FB05200294694600070196009503940A
:10B1A000FCF7ACFA0520012229460007FCF767FBF3
:10B1B0001A48007800281CD1194C2068C10718D102
:10B1C000184D2968884214D0174801781748142967
:10B1D00001D3FF2101E0FF21090201601449006849
:10B1E0000B6814490A681449096800F00DFC2068CE
:10B1F000286012A0FEF752FA05B0F0BDA8040020A6
:10B20000CC0600202407002034050020BC050020C7
:10B210004406002000100240007000403000002072
:10B2200028000020340000203800002024000020E6
:10B23000180000201C0000202000002077616B75A2
:10B240002075700D0A000000F0B587B003F0CCFC4B
:10B250006B4800F099FB6B4EF0806948801C00F051
:10B2600093FB30816648001D00F08EFB664D7081B7
:10B27000FF20023068802C464034E18CE120000140
:10B28000002900D1E084217971700491E0846887FD
:10B290005E49E88E08705E49E88F08705D49A88FA6
:10B2A0000870A07930705C49A87A08705B48AF8854
:10B2B00007605B4805210180E8880390F9F718FFD3
:10B2C0005849088001463846F9F712FF88000818E7
:10B2D00087B2554807807D20C0007843FAF74CFAC2
:10B2E000524A534BFAF79EF9FAF78CFA514980B259
:10B2F000088000905048078050480188C820F9F71E
:10B30000F7FE4F49012208804E480027028003982B
:10B31000B0807D200499C000002904D13C49B08050
:10B320000A703C490F70B188F9F7E2FE4349088082
:10B3300045494648009AFCF701FC002801D072B646
:10B34000FEE7A08C012804D0608C414E012838D043
:10B3500040E0FF20000203461A46114600F054FB6D
:10B36000FF25F5352846FCF791F8FF200004034639
:10B370001A46114600F048FB2846FCF787F80023E0
:10B380001A461946184600F03FFB2846FCF77EF89F
:10B3900030486946088072B680212F4D2846FBF759
:10B3A00081FA002804D0022269462846FBF720FBD8
:10B3B00062B6A78403F080FC642002F077FE02F0FE
:10B3C000ABF867842F8003F077FC642002F06EFEF8
:10B3D0002248C660208C012807D1278403F06CFC2A
:10B3E000642002F063FE1D48C66028881C4988421C
:10B3F00002D1E888002801D11848C66007B0F0BD26
:10B40000004F00080000002064070020B801002061
:10B410007400002075000020620000205C00002005
:10B42000660000206800002064000020F853E3A5B7
:10B430009B843E406A0000206E0000206C000020CB
:10B440007800002076000020FF7F00000405002027
:10B450000400FA05AAAA0000384A000800ED00E03E
:10B46000AA55000000B5044940208862FF20F5304D
:10B4700003F03EFC00BD000000040050FF23024624
:10B480001B0200B519020D489A4202D100F0C0F823
:10B4900000BD8A4202D100F057F809E0FF2A04D02B
:10B4A000824205D100F002F900BD00F009F800BDAC
:10B4B000002AFCD100F07AF800BD0000FFFFFF0079
:10B4C00000B500F02FF800F02DF800F02BF800F098
:10B4D00029F800F027F800F025F800F023F800F034
:10B4E00021F800F01FF800F01DF800F01BF800F044
:10B4F00019F800F017F800F015F800F013F800F054
:10B5000011F800F0B7F800F0B5F800F0B3F800F06B
:10B51000B1F800F0AFF800F0ADF800F0ABF800F0D3
:10B52000A9F800BD07484021816100BF00BF00BFEE
:10B5300000BF00BF00BF816200BF00BF00BF00BFEF
:10B5400000BF70470004005000B500F093F800F011
:10B5500091F800F08FF800F08DF800F08BF800F013
:10B5600089F800F087F800F085F8FFF7DBFFFFF7B8
:10B57000D9FFFFF7D7FFFFF7D5FFFFF7D3FFFFF79F
:10B58000D1FFFFF7CFFFFFF7CDFFFFF7CBFFFFF7AF
:10B59000C9FFFFF7C7FFFFF7C5FFFFF7C3FFFFF7BF
:10B5A000C1FFFFF7BFFFFFF7BDFF00BD00B5FFF70D
:10B5B000B9FFFFF7B7FFFFF7B5FFFFF7B3FFFFF7DF
:10B5C000B1FFFFF7AFFFFFF7ADFFFFF7ABFFFFF7EF
:10B5D000A9FFFFF7A7FFFFF7A5FFFFF7A3FFFFF7FF
:10B5E000A1FFFFF79FFFFFF79DFFFFF79BFFFFF70F
:10B5F00099FFFFF797FFFFF795FFFFF793FFFFF71F
:10B6000091FFFFF78FFFFFF78DFFFFF78BFF00BD67
:10B6100000B5FFF787FFFFF785FFFFF783FFFFF711
:10B6200081FFFFF77FFFFFF77DFFFFF77BFFFFF74E
:10B6300079FF00F01FF800F01DF800F01BF800F093
:10B6400019F800F017F800F015F800F013F800F002
:10B6500011F8FFF767FFFFF765FFFFF763FFFFF7DD
:10B6600061FFFFF75FFFFFF75DFFFFF75BFFFFF78E
:10B6700059FF00BD0C484021816100BF00BF00BFE1
:10B6800000BF00BF00BF00BF00BF00BF00BF00BFC2
:10B6900000BF00BF00BF00BF816200BF00BF00BF8E
:10B6A00000BF00BF704700000004005000B5FFF766
:10B6B000E1FFFFF7DFFFFFF7DDFFFFF7DBFFFFF73E
:10B6C000D9FFFFF7D7FFFFF7D5FFFFF7D3FFFFF74E
:10B6D000D1FFFFF7CFFFFFF7CDFFFFF7CBFFFFF75E
:10B6E000C9FFFFF7C7FFFFF7C5FFFFF7C3FFFFF76E
:10B6F000C1FFFFF7BFFFFFF7BDFFFFF7BBFFFFF77E
:10B70000B9FFFFF7B7FFFFF7B5FFFFF7B3FF00BDC6
:10B7100008B5002808D00246002106480091044BD5
:10B720000068FEF743F908BD002000F005F808BDE9
:10B7300039B700089C010020044972B60248C8606D
:10B74000BFF34F8F704700000400FA0500ED00E0E2
:10B75000F8B56E4C00256E48E570C1887D20C000AC
:10B76000F9F7C6FC6B4E01463080C820F9F7C0FCE3
:10B7700069490880A07A401CA072C00706D0E08BFF
:10B78000411EE183022801D2C820E0830A2002F092
:10B7900096FF7D20400102F0ADFF604F2020BD727A
:10B7A00078725B48C1887D20C000F9F7A1FC7873EE
:10B7B0005B4856490078B8733846203113380A7808
:10B7C00002754978417552491E308A780270C978ED
:10B7D0004170411C4E482030027ECA70407E087184
:10B7E0004B482230027E4A71407E887100220C391B
:10B7F000172003F04FF80021172003F05DF8022016
:10B8000002F0AEFF474F01E0FEF736FC00210F20AB
:10B8100002F0C2FE38422063F6D0206B411C73D088
:10B8200040046FD58122D20100210F2003F007F8D8
:10B830000021102002F0B0FE41063848490E0022D7
:10B84000B430A16402F0F8FE344FB437787A11288E
:10B8500058D102223449781DF9F7CFFC002851D184
:10B86000F81F027A69460A70407A4870B97A3180C6
:10B87000C820F9F73DFC28492C4E0880387BE0832E
:10B8800038462838C08E308038462838008FA0834C
:10B890002748FCF74FF96084A08B2649FF30C3305E
:10B8A00080B2A08388420BD949424018A0833088D7
:10B8B0002049401C80B20B313080884200D3358053
:10B8C00030887D21C9004843A18B40182064684618
:10B8D000008820841149B87CC73120714200084695
:10B8E0000E469130F9F74AFC207931464200124861
:10B8F000F9F744FCE08BFF2804D025730220207068
:10B90000FBF736FAF8BDFFE701F014FEA0000020B7
:10B91000640700206C00002078000020A00C0020AC
:10B92000B801002000D027245C0000206000002027
:10B9300004050020E7030000100E002070B586B05B
:10B9400014216846F9F733FC0E4E002201213046DF
:10B95000FBF795FF012500240095029469463046C7
:10B9600001950394FBF7CAFE0320019002946946F7
:10B97000009503943046FBF7C1FE022002F096FBCF
:10B9800006B070BD0004005000887047704700008A
:10B99000F8B5044600206A461080194D55222A70D9
:10B9A000AA226A700322AA70661DEE702A7169715C
:10B9B000144A49008918AC712246E81DF9F7DEFBEC
:10B9C000002007E029186A468978128889186A4693
:10B9D0001180401CB042F5DB611DA81CFAF7E8FCA1
:10B9E00001466846018029190078C8716846407888
:10B9F0000872224609320249002001F0A3FBF8BD7B
:10BA0000C80B002064070020F8B5164604460F4610
:10BA1000012205201D46D1030007FBF730FFFFF789
:10BA200021FD2846FFF72AFD3046FFF727FD38465F
:10BA3000FFF724FD2046FFF721FDFFF713FDF8BDBA
:10BA400010B5012105200022C9030007FBF717FFED
:10BA500010BD0000FFB505468400114881B01E46A8
:10BA6000201804220A9FF9F789FB0D4804222C3084
:10BA700020180399F9F782FB094809495830201822
:10BA800006606800B03140183978017079784170EB
:10BA900004480349006D8431085105B0F0BD000031
:10BAA000FC0E0020A000002010B5FAF799FBFDF76E
:10BAB0009BFE00280DD0FDF797FE0B24E401001932
:10BAC0000069002805D0FDF78FFE0019016902A06A
:10BAD0008847002010BD00004F4B0D0A00000000F9
:10BAE00010B5FAF79BFBFDF77FFE00280DD0FDF7A0
:10BAF0007BFE0B24E40100190069002805D0FDF746
:10BB000073FE0019016902A08847002010BD0000E3
:10BB10004F4B0D0A0000000010B5022814DAFDF7A3
:10BB200063FE00280DD0FDF75FFE0B24E401001931
:10BB30000069002805D0FDF757FE0019016907A02C
:10BB400088470020C04310BD4868F9F763FB002810
:10BB500001D1FDF7ADFC002010BD000064656275E9
:10BB6000675F6F666620666C61670D0A0000000003
:10BB700010B5022814DAFDF737FE00280DD0FDF7C6
:10BB800033FE0B24E40100190069002805D0FDF7FD
:10BB90002BFE0019016907A088470020C04310BD93
:10BBA0004868F9F737FB002801D1FDF787FC002032
:10BBB00010BD000064656275675F6F6E20666C6122
:10BBC000670D0A0010B5FFF765FAFDF70DFE0028B6
:10BBD0000DD0FDF709FE0B24E401001900690028CF
:10BBE00005D0FDF701FE0019016902A08847002079
:10BBF00010BD00004F4B0D0A0000000010B5FFF70C
:10BC000055FAFDF7F1FD00280DD0FDF7EDFD0B24F1
:10BC1000E40100190069002805D0FDF7E5FD0019D1
:10BC2000016902A08847002010BD00004F4B0D0A9B
:10BC30000000000070B5FDF7D7FD0B25ED010028D1
:10BC40000CD0FDF7D1FD40190069002806D0FDF7A2
:10BC5000CBFD401902690FA111A09047FDF7C4FD6B
:10BC6000002815D0FDF7C0FD4019006900280FD04D
:10BC7000FAF752FAF9F7E4FD04460E46FDF7B4FD73
:10BC8000401905690B482246017833460AA0A847A7
:10BC9000002070BD76312E302E302E340000000092
:10BCA00056657273696F6E3A20202020202025731C
:10BCB0000D0A000038000020426174746572793A00
:10BCC0002020202020202575252520252E3266566F
:10BCD0000D0A000010B511210248FDF74FFD0020AC
:10BCE00010BD000048ED00080020704710B507287F
:10BCF00014D0FDF779FD00280DD0FDF775FD0B245C
:10BD0000E40100190069002805D0FDF76DFD001958
:10BD1000016903A088470020C04310BD002010BD6A
:10BD200075736167653A207274635F736574207917
:10BD3000797979206D6D206464206868206D6D20AC
:10BD400073730D0A0000000010B50020FFF7E0FC3F
:10BD5000002010BD10B50B24E401062812DAFDF70F
:10BD600043FD00280BD0FDF73FFD001900690028B6
:10BD700005D0FDF739FD001901690BA088470020A7
:10BD8000C04310BDFDF730FD00280BD0FDF72CFDA2
:10BD900000190069002805D0FDF726FD001901698A
:10BDA00011A08847002010BD7365745F6164632033
:10BDB0006E6F726D616C5F6D696E206E6F726D611A
:10BDC0006C5F6D6178206572726F725F6D696E2055
:10BDD0006572726F725F6D6178206572726F725FEB
:10BDE000636E740D0A0000004F4B0D0A0000000046
:10BDF00010B50B24E40102280FDAFDF7F5FC00284A
:10BE00001BD0FDF7F1FC00190069002815D0FDF7E3
:10BE1000EBFC001901690AA00EE0FDF7E5FC002823
:10BE20000BD0FDF7E1FC00190069002805D0FDF7F3
:10BE3000DBFC0019016904A08847002010BD000048
:10BE40004552524F520D0A004F4B0D0A00000000A0
:10BE500070B500250B24ED43E40102280FDAFDF74D
:10BE6000C3FC002822D0FDF7BFFC001900690028A0
:10BE70001CD0FDF7B9FC0019016916A015E048684F
:10BE8000F9F7C8F9002801D0082811D9FDF7ACFC52
:10BE900000280BD0FDF7A8FC00190069002805D088
:10BEA000FDF7A2FC001901690EA08847284670BD65
:10BEB000FDF79AFC00280BD0FDF796FC00190069ED
:10BEC000002805D0FDF790FC0019016908A08847FB
:10BED000002070BD7365745F6465765F6964206976
:10BEE000640D0A006964206572726F720D0A0000A9
:10BEF0004F4B0D0A0000000010B50B24E40103288D
:10BF000012DAFDF771FC00280BD0FDF76DFC00196B
:10BF10000069002805D0FDF767FC001901690BA036
:10BF200088470020C04310BDFDF75EFC00280BD001
:10BF3000FDF75AFC00190069002805D0FDF754FCF4
:10BF4000001901690AA08847002010BD7365745F5D
:10BF50006970205B7365727665725F69705D205BE6
:10BF60007365727665725F706F72745D0D0A0000A2
:10BF70004F4B0D0A0000000010B50B24E40103280C
:10BF800012DAFDF731FC00280BD0FDF72DFC00196B
:10BF90000069002805D0FDF727FC001901690BA0F6
:10BFA00088470020C04310BDFDF71EFC00280BD0C1
:10BFB000FDF71AFC00190069002805D0FDF714FCF4
:10BFC000001901690AA08847002010BD7365745FDD
:10BFD00077696669205B737369645D205B70617368
:10BFE00073776F72645D205B69705D0D0A000000FD
:10BFF0004F4B0D0A0000000010B5FFF76BF8002052
:10C0000010BD10B5FEF722FB002010BD034A1168D9
:10C01000382389B2994301431160704700300140D1
:10C0200070B5104C2078002811D00025012806D0CA
:10C0300002280FD0032801D1FEF76EFD70BDFFF777
:10C0400087FB607B411C617309E0257070BDFAF7C6
:10C0500041FA70BDFAF78CFE207B411C2173052844
:10C06000F3D870BDA000002010B5FDF7CBFCFBF7A6
:10C0700021FC10BD10B59AB034216846F9F797F845
:10C08000142115A8F9F793F820210DA8F9F78FF8D6
:10C09000234801680324E402A143C2148918016003
:10C0A000FBF7E6FD1F480169214301610E20009066
:10C0B000FF200130029010200490022009904004DB
:10C0C00001210B900001059100240C9003910A942A
:10C0D0006846FCF741F8002801D072B6FEE70F2051
:10C0E000159003201690179418940121199415A8FF
:10C0F000FBF7C4FE002801D072B6FEE787200D9042
:10C1000003200F9480041490109411940DA8FBF751
:10C11000EBFD002801D072B6FEE71AB010BD00009A
:10C12000007000404010024002490148886070479A
:10C130000050000800ED00E0F0B402680124A407FC
:10C14000144D154E154FA04205D0A84203D0B04261
:10C1500001D0B84203D170239A434B681A43A042DE
:10C1600005D0A84203D0B04201D0B84204D1032385
:10C170001B029A43CB681A4380239A430B691A43E4
:10C1800002608A68C2620968816201214161F0BC73
:10C190007047000000040040000801400014014006
:10C1A00010B4C906C90E01238B40046A9C43046283
:10C1B000036A8A401343036210BC704730B484683A
:10C1C000FF252D02AC431B0213430B432343836023
:10C1D00030BC7047826870239A430A4307210A43A0
:10C1E0008260704730B4026A520852000262026AEA
:10C1F000446883697025AB439B089B000D681D4311
:10C2000002239A438B681343446085614968416304
:10C21000036230BC704730B4026A10239A43026252
:10C22000036A4568826907242403A2430324240285
:10C23000A2430C6824021443202293438A6812010B
:10C240001A434560846149688163026230BC70476B
:10C2500030B4026AFF2301339A430262026A4468DF
:10C26000C3697025AB439D08AD000B682B430125C6
:10C270006D02AA438D682D0215434460C36149686D
:10C28000C163056230BC704730B4026A01231B03EE
:10C290009A430262036A4568C26907242403A243E1
:10C2A00003242402A2430C682402144301225203F3
:10C2B00093438A6812031A434560C4614968016464
:10C2C000026230BC704730B4036A046A64086400D8
:10C2D00004628469F025AC43120122430A24A3437B
:10C2E0000B438261036230BC704730B4036A102490
:10C2F000A34303628369046A0F252D03AB43120332
:10C300001A43A0239C43090121438261016230BC8E
:10C310007047000070B5FF24114D0134AC62AF20AE
:10C32000800001F0CAFEAC6102F064F90D4C0E4DC4
:10C33000A06007E002F05EF9A060FDF79DFE606876
:10C34000401C6060A068A842F4D102F037F80020D9
:10C350006060FFF765FE02F031F802F017F870BD7B
:10C36000000400507C0000203001CADE10B50548F2
:10C370000549806A884204D3642001F097FE01F0E9
:10C38000CBF810BD000000200094357710B4818CEC
:10C39000C90707D001684A6801235B049A43836A8E
:10C3A0001A434A60818C890707D501684A680123CE
:10C3B0001B049A43C36A1A434A60818C490707D514
:10C3C00001684A6801239B049A43036B1A434A603D
:10C3D000818C090707D501684A680123DB039A436A
:10C3E000436B1A434A60818CC90607D501688A6885
:10C3F00001231B039A43836B1A438A60818C89064D
:10C4000007D501688A6801235B039A43C36B1A430B
:10C410008A60818C490612D501684B680122120599
:10C42000046C934323434B60016C914207D1016834
:10C430004A6803235B059A43436C1A434A60818C24
:10C44000090607D501684A680123DB04806C9A431A
:10C4500002434A6010BC7047F0B583B004462646DC
:10C46000002780367760FBF711FA02902068006899
:10C4700025460007603500281CDA2A480090012173
:10C48000002249052046029B00F09AFC002811D0AA
:10C49000EFF31081012080F3108820680268802368
:10C4A0009A43026081F310882020E0672F760320F2
:10C4B00003B0F0BD20680068400729D519480090F6
:10C4C0000121002289052046029B00F079FC00280A
:10C4D0001ED0EFF31081012080F3108820680268DD
:10C4E000FF2321339A43026081F31088EFF3108118
:10C4F000012080F310882068826852085200826010
:10C5000081F31088202030602F76032003B0F0BD27
:10C510002020E0673060276667662F76002003B032
:10C52000F0BD0000FFFFFF0110B5806A0022014648
:10C5300040314A834A82FCF7FBFB10BDF8B5846AA0
:10C54000E06F254680352E68216889680027090636
:10C55000002906DA212804D152200753204600F092
:10C56000DFF820688068400606D5222E04D15A20C4
:10C570000753204600F090F868681021084368606F
:10C580002046FCF7D5FBF8BD70B50146886A0968FE
:10C59000096800238906002937DB5A210B52EFF383
:10C5A0001082012181F3108801680C68FF25013594
:10C5B000AC430C6082F31088EFF31082012181F309
:10C5C000108801688C68640864008C6082F31088AD
:10C5D000EFF31082012181F3108801688C684025F7
:10C5E000AC438C6082F31088202280210A50016EB7
:10C5F00001290AD1EFF3108281F3108801680C68D9
:10C600001025AC430C6082F310884366016E01294B
:10C6100002D0FCF733FE70BD5821095AFCF764FBC9
:10C6200070BD10B5806A01214166016E012902D0FA
:10C63000FCF728FE10BD5821095A4908FCF754FBA5
:10C6400010BD10B50146886A0968096889061BD4BF
:10C65000002252210A52EFF31082012181F3108847
:10C6600001688B688024A3438B6082F31088EFF30A
:10C670001081012282F310880068026840231A4367
:10C68000026081F3108810BDFCF70CFF10BD10B5DF
:10C69000806AFCF70BFF10BD10B4EFF3108201218C
:10C6A00081F3108801680B68FF242134A3430B60D9
:10C6B00082F31088EFF31082012181F31088016862
:10C6C0008B685B085B008B6082F31088016E012928
:10C6D0000AD1EFF3108281F3108801680B681024EF
:10C6E000A3430B6082F31088202280210A5000218E
:10C6F0000166816610BC704710B5EFF3108201210E
:10C7000081F3108801680B684024A3430B6082F317
:10C7100010882021C1670021C166FCF7C3FE10BD4F
:10C7200010B4EFF31082012181F3108801680B68C7
:10C73000C024A3430B6082F310882021C16710BC82
:10C740007047000070B5014640318B8B0246803245
:10C75000156814460268222D04D090690821084308
:10C76000906170BD526A456D1A402A80426D921CDC
:10C7700042654A8B521E4A834A8B002AF1D1EFF35D
:10C780001083012282F3108802681568FF26213683
:10C79000B543156083F31088EFF31083012282F311
:10C7A0001088026895686D086D00956083F31088A5
:10C7B00020222260002484664466184B02689A4254
:10C7C0000ED053681B020BD5EFF31083012585F3C0
:10C7D000108815680126B606B543156083F31088E6
:10C7E000026E012A02D0FCF749FD70BD0466EFF32A
:10C7F0001083012282F31088026815681024A54373
:10C80000156083F310880268D369DB43DB0600D42C
:10C810001462098BFCF768FA70BD00000048004004
:10C8200070B5014640318B8B024680321568144644
:10C830000268222D04D0906908210843906170BDE0
:10C84000526A1A40436D1A70426D521C42654A8BFF
:10C85000521E4A834A8B002AF1D1EFF31083012242
:10C8600082F3108802681568FF262136B5431560EB
:10C8700083F31088EFF31083012282F3108802689B
:10C8800095686D086D00956083F310882022226002
:10C89000002484664466184B02689A420ED053689E
:10C8A0001B020BD5EFF31083012585F31088156863
:10C8B0000126B606B543156083F31088026E012A7F
:10C8C00002D0FCF7DBFC70BD0466EFF3108301229D
:10C8D00082F31088026815681024A543156083F35D
:10C8E00010880268D369DB43DB0600D41462098B2D
:10C8F000FCF7FAF970BD000000480040F8B50446A6
:10C900000025904F20682269A168E369114362699C
:10C910001A43114302688C4B1A400A430260206894
:10C920004168032212039143E26811434160A06908
:10C930002168B94201D0226A10438A680B231B0286
:10C940009A4302438A608149226881488A4213D10E
:10C95000C0688007800F07D0012809D0022805D0C1
:10C96000032807D0102142E0012140E002213EE0EF
:10C9700004213CE008213AE076498A4213D1C0689C
:10C980000C21084007D0042809D0082805D00C281D
:10C9900007D010212BE0002129E0022127E004210B
:10C9A00025E0082123E06C498A4201D100211EE0E4
:10C9B0006A498A4201D1002119E0BA4216D1C06801
:10C9C0000321890208400BD001218902401A0BD0B3
:10C9D000401A07D0884201D1082108E0102106E062
:10C9E000002104E0022102E0042100E010215D4862
:10C9F0005B4E8300BA4236D1002913D0022914D0ED
:10CA0000042917D0082918D000200125002861D05A
:10CA1000626851005118814202D8110381420FD23D
:10CA2000012589E0FBF72EFBF0E73168C906EDD45C
:10CA30001846EBE7FBF746FBE8E70120C003E5E714
:10CA4000010E06025008002330185941F8F766FB22
:10CA500003210902444A411A914202D82168C86060
:10CA60006AE0012568E00122E769D203974234D1E8
:10CA7000092919D20F007F443F79FF19BF440407E9
:10CA80000A140F1414141200FBF7FCFA0EE0FBF763
:10CA900009FB0BE03168C90608D4184606E0FBF72D
:10CAA00011FB03E0104601E000200125002843D0DF
:10CAB000616840004A088018F8F71AFB02462B49C3
:10CAC000103A8A4207D8491C01400007420F0A4326
:10CAD0002068C26030E001252EE0092919D20F003C
:10CAE0007F443F79FF19BF4404070A140F1414143C
:10CAF0001200FBF7C7FA0EE0FBF7D4FA0BE031683F
:10CB0000C90608D4184606E0FBF7DCFA03E0104635
:10CB100001E00020012500280ED061684A081018A5
:10CB2000F8F7E6FA0146114A1039914203D8216814
:10CB300080B2C86000E001250020A066E0662846BB
:10CB4000F8BD000000480040F369FFEF00380140E5
:10CB50004010024000440040004C004000500040A3
:10CB60000010024000093D00FFFC0F00EFFF000035
:10CB700070B5044661655820025300212546803572
:10CB8000696022202860606F002819D0214BC362A1
:10CB9000636F21481863636F20485863606F816337
:10CBA0002168666D134624313246606FFAF735FC12
:10CBB000002805D01020686020202860012070BD6A
:10CBC000206900280CD0EFF31081012080F3108839
:10CBD00020680268FF2301331A43026081F3108842
:10CBE000EFF31081012080F3108820688368012210
:10CBF0001343836081F31088EFF3108182F3108870
:10CC00002068826840231A43826081F310880020E4
:10CC100070BD000089C5000823C600083DC5000896
:10CC200070B44165014640310A834A83002484661A
:10CC3000012382681B03FF259A4207D10269002A5B
:10CC400001D08D8319E02B4A8A8316E07F26002AC3
:10CC500009D001252D07AA420ED10269002A09D068
:10CC60003F228A8309E00269002A01D08E8304E012
:10CC70008D8302E08E8300E08C83014680314C601E
:10CC800022220A60EFF31082012181F310880168EB
:10CC90008C6801252C438C6082F31088816899424E
:10CCA00002D10169002912D0134981660169002966
:10CCB00010D0EFF31081012282F31088006802681F
:10CCC000FF2321331A43026081F310880EE00B49E1
:10CCD0008166EBE7EFF31081012282F31088006890
:10CCE000026820231A43026081F3108870BC002080
:10CCF00070470000FF01000021C8000845C7000878
:10CD000010B4C16F212910D1014640314A8A002A4E
:10CD10000DD0C26C03681288D205D20D9A62C26C23
:10CD2000921CC264488A401E488210BC7047EFF3D0
:10CD30001082012181F3108801680B688024A343CD
:10CD40000B6082F31088EFF31081012282F31088C8
:10CD50000068026840231A43026081F3108810BC07
:10CD6000704710B4C16F21290ED1014640314A8A63
:10CD7000002A0BD0C26C036812789A62C26C521CF3
:10CD8000C264488A401E488210BC7047EFF310828C
:10CD9000012181F3108801680B688024A3430B6094
:10CDA00082F31088EFF31081012282F3108800686B
:10CDB000026840231A43026081F3108810BC704758
:10CDC000FFB583B00C9D04460E4617462068C16926
:10CDD0003046884327D00020B84245D120468030D5
:10CDE000029020380190681C36D0FAF74FFD069962
:10CDF000401AA84219D8002D17D0206801684907A9
:10CE00002AD5C169C943090712D4206808250562DB
:10CE10002046FFF741FC0298456001990020087602
:10CE2000012007B0F0BD0120D6E7032007B0F0BD18
:10CE3000C069C04300050FD401202168C002086208
:10CE40002046FFF729FC029820214160019900202B
:10CE50000876032007B0F0BD2068C16930468843DA
:10CE600005D00020B842BED0002007B0F0BD0120A0
:10CE7000F8E7000010B50248FBF75EFF10BD0000A8
:10CE8000BC05002010B50248FBF756FF10BD00009E
:10CE900044060020F8B51D4D0E0034D0032832D2D0
:10CEA000742148431A494418A078002802D0012868
:10CEB00022D028E0E168A068421860680090406FC6
:10CEC000006840682769101A0818C01BF8F710F9A5
:10CED000012905D817D100980068C069800612D4CE
:10CEE0003878307061692069884201D1A06800E01B
:10CEF000401C2061002506E0204618303146FCF732
:10CF000023FB0028F6D02846F8BD0000FFFFFFFFF6
:10CF1000B42C002070B50C00064601D0032E02D3BD
:10CF20000020C04370BD7421484321490E5422782B
:10CF300045186A706078A8706068A860A168E960A8
:10CF40006278002A02D0012A05D00BE0286140183F
:10CF5000401E686106E0284618300123A268616817
:10CF6000FCF7CDFAE068E86220692863A0692867C9
:10CF7000606968632078002801D0012806D1214625
:10CF80000C310EC928463830FCF74BFF607800287A
:10CF900004D0012806D0022804D006E0304600F074
:10CFA00009F802E0304600F021F8002070BD0000D2
:10CFB000B42C002038B50C497422504342185068F4
:10CFC000016804E04C6A6B461C801C881C80CB699D
:10CFD0001B07F7D491681161D368CC18641E5461A3
:10CFE0009AB2FCF7E3F838BDB42C00207421484312
:10CFF000044910B540180146683140680122FCF729
:10D0000009F910BDB42C002070B5054674201A49EA
:10D0100068434418A078002802D0012807D00DE00A
:10D02000A0682061E1684018401E606106E020466B
:10D0300018300123E268A168FCF761FA60780028E3
:10D0400001D0012806D121462C310EC920463830A6
:10D05000FCF7E7FEA078002804D0012806D00228BB
:10D0600004D006E02846FFF7A5FF02E02846FFF7B8
:10D07000BDFF002070BD0000B42C002070B50D0075
:10D0800001D0032802D30020C04370BD742148435F
:10D090000449441874212046FCF7E4FC0020656034
:10D0A00070BD0000B42C002010B502460E490020CF
:10D0B000742343435B185B6893420FD1742242434D
:10D0C00051188978002906D0012901D0022901D1FF
:10D0D000FFF78CFF10BDFFF76DFF10BD401CC0B205
:10D0E0000328E5D310BD0000B42C002038B501465C
:10D0F0001348002474226243121852688A4219D1DC
:10D10000742161430818817801290BD0022908D1C4
:10D11000016F002902D0806EC0B288472046FFF719
:10D1200065FF38BD816E6A46117069461830FCF79C
:10D13000CBF9F3E7641CE4B2032CDBD338BD000069
:10D14000B42C0020F7B582B0002100910399154658
:10D15000002903D0002D01D0032803D30020C043B1
:10D1600005B0F0BD742148432B4946187078344609
:10D170003834002804D0012820D0022842D049E0C9
:10D18000FCF7C6FA20462946FCF71DFE070033D0FF
:10D1900020463946FCF7E3FD2A4638680399F7F73D
:10D1A000EDFF2046FCF7F1FD0446FCF73FFCA088AC
:10D1B000216882B27068FCF7D7F82BE0FCF7A8FA78
:10D1C00020462946FCF7FFFD070015D020463946CA
:10D1D000FCF7C5FD2A4638680399F7F7CFFF2046CC
:10D1E000FCF7D3FD0446FCF721FCA088216882B23D
:10D1F0007068FCF713F90DE0FCF718FC0020C04341
:10D20000009007E0134664204343AAB27068039974
:10D21000FCF739F80098A3E7B42C002070B51F4A3A
:10D22000002174234B439B185B68834231D17420E7
:10D2300041438C186078002816D0012813D120466D
:10D2400038300546FCF7A1FD01462846FCF771FD84
:10D250002846FCF79AFD002805D081888AB201682B
:10D260006068FCF7DBF870BD204638300546FCF7F7
:10D270008CFD01462846FCF75CFD2846FCF785FD41
:10D280000028F0D081888AB201686068FCF76CF8E9
:10D2900070BD491CC9B20329C3D370BDB42C002092
:10D2A000F8B53E4C002321783D4A1D46082910D090
:10D2B000072947D0062950D0052952D0042953D038
:10D2C000032954D0002956D0012958D002295AD018
:10D2D0005BE0A17800264A1F04E0314FBF5DFB18D8
:10D2E0009BB2761C9642F8DB667927799A19511819
:10D2F000E3786278C9188918C9194018C043000634
:10D30000000E1AD1012E14D0022E16D12548244920
:10D31000C018F7F733FF01F0CFFC642000F0C6FE21
:10D32000BFF34F8F21492048C860BFF34F8F00BF24
:10D33000FDE759081046FEF72BFB2570E570A57038
:10D34000A571F8BDA1795054491CC8B2A071A1784B
:10D35000491F8842F5D1082001E060700720207045
:10D36000F8BDE0700620FAE760710520F7E7A070CD
:10D37000E5700420F3E7552807D10120EFE7AA283C
:10D3800003D10220EBE7032803D02570E570A570D8
:10D39000F8BD032020702071F8BD0000930000202C
:10D3A000640B0020640700200400FA0500ED00E093
:10D3B00070B5194C206B00282DD12169A06A401A44
:10D3C0000A2828D3FF23A361E269216A606AFEF775
:10D3D0001BFBFEF79FFFA06A2061A0890F4D401C38
:10D3E00080B2A08129780026032901D3A68106E016
:10D3F000052804D9032902D20120A07000E0A670FC
:10D4000007A0FCF74BF92E70A6613346E269216A4A
:10D41000606AFEF7F9FA70BD00000020AB00002042
:10D42000D3D0D0A7B2E2BEE025640D0A0000000010
:10D4300070B50D48FAF77EFB0C4C01252082AD0338
:10D4400009E00948FAF776FB80B22082A189FF390A
:10D450002D39884206DBA18980B28842F1D349196F
:10D460008842EED870BD000004050020280100208D
:10D470007CB51546024600201C4600290BD0491EEB
:10D4800000920191044B6A462146284600F002FAB8
:10D49000009A002111707CBDCDDF00082021020C14
:10D4A00001D010211046020A01D0104608390209A5
:10D4B00001D01046091F820801D01046891E42087B
:10D4C00001D0881E7047081A7047F0B4040C8BB264
:10D4D000264682B25E430D0C1046370C5843360484
:10D4E00080190021794116466E43370C36048019A5
:10D4F000794126466E438919F0BC704730B47446B2
:10D50000641E2578641CAB4200D21D46635D5B003F
:10D51000E31830BC18470000BFF34F8F044903489D
:10D52000C860BFF34F8F00BFFDE700000400FA059D
:10D5300000ED00E0BFF34F8F04490348C860BFF31C
:10D540004F8F00BFFDE700000400FA0500ED00E08A
:10D55000BFF34F8F04490348C860BFF34F8F00BF2C
:10D56000FDE700000400FA0500ED00E00048704708
:10D57000A404002002E008C8121F08C1002AFAD142
:10D5800070477047002001E001C1121F002AFBD143
:10D59000704708B50021684601706B4601220221E0
:10D5A0002C2001F05BF90221684601706B460122D4
:10D5B0002C2001F053F908BD38B504466D206946AA
:10D5C00008706B46012207492E2001F047F90649F1
:10D5D000002C01D0054A00E0054A2E2001F024F974
:10D5E00038BD00000608000006180000070600000D
:10D5F0000716000038B504466B460222002136208B
:10D6000000F0FEFFB3212300FFF778FF0E0F08158F
:10D610003A3A3A3A1C273A3A2F34483A00216846B7
:10D62000017040784108490014E069460878800894
:10D630008000401C04E06946087880088000801C57
:10D6400008701DE0684602780A404832027041784E
:10D65000802001436846417012E0684602780A4023
:10D66000027040784106490EF4E769464878022185
:10D67000084303E069464878FD2108406946487040
:10D680006B4601220021362001F0E8F8012200ABB0
:10D6900011463620013301F0E1F838BD69460878BB
:10D6A000CF21084069462030CAE708B50321684603
:10D6B0004170012101706B4602220021362001F0E9
:10D6C000CDF80122D20306212D2001F0ADF8012072
:10D6D00000F0ECFC0120FFF78DFF08BD08B5020A41
:10D6E00069464A7008706B46022204212D2001F021
:10D6F000B5F80320694608706B46012206212D20EB
:10D7000001F0ACF80020694608706B460122062142
:10D710002D2001F0A3F80A212D2000F03DFF08BDC7
:10D72000F0B51FB486B00998089A030D0021024392
:10D7300014D05148514A1818504305141198012823
:10D7400010981AD0281A401C00264D4F4D490096BB
:10D7500001910490002812DA444211E0119801244A
:10D7600049A3012801D11098C1430698119A8460F9
:10D770000360C26041600BB0F0BD4042E4E7044684
:10D78000210500203F4A001C51410391029012E004
:10D79000E00707D032463B4601990098F7F7DAFEDA
:10D7A0000191009032463B4610461946F7F7D2FEEB
:10D7B00006460F466410002CEAD10498039B00280B
:10D7C000029A0999089806DAF7F7C4FE019B009AB5
:10D7D000F7F7C0FE05E0F7F725FF019B009AF7F782
:10D7E00021FF04460E460022284BF8F751F803D8D3
:10D7F0000020C043014607E00022254B2046314669
:10D80000F7F7F6FDF8F780F9102409E0002C0ADBA1
:10D810000A220023F7F782FC079B30321A55641E58
:10D8200002460A43F2D11122641C079B121B1C19E9
:10D83000119B012B03D0012308430ED10AE00843BA
:10D8400004D0112010900020119077E71098151A3D
:10D850006D1E0BE01098824202DD00236D1C03E078
:10D86000824201DA00236D1E002BEED0069811993A
:10D870008260C16030C07EE701FCFFFF104D0000F8
:10D88000000014400000F03F300000000000F043B2
:10D890000000E03FFFB597B00646002518E22528B6
:10D8A00077D100242746FD49049400E00443761C08
:10D8B00032780120203A90400842F7D130782A2867
:10D8C0000ED00222307801463039092916D8049941
:10D8D0000A235943303940181443761C0490F1E769
:10D8E000189802C804911890002904DA0120400316
:10D8F00004434842049002200443761C30782E28CA
:10D9000014D1042004437078761C2A2809D1189871
:10D91000761C80C8189009E00A214F43303FC71990
:10D92000761C3078014630390929F5D930786C28D1
:10D9300010D006DC4C281AD068280ED06A2817D1DF
:10D9400004E0742813D07A2812D110E00120400599
:10D9500004430CE00121090501E0032109050C4302
:10D960007178814203D1012000052418761C761CB1
:10D970003078119066280BD013DC58287DD009DC54
:10D9800000287BD04528F6D04628F4D047281AD165
:10D99000A5E118E0632835D0642870D0652812D13D
:10D9A0009DE170286CD008DC6728F1D069287BD015
:10D9B0006E280DD06F2806D1BAE073282ED07528B6
:10D9C00071D0782859D01A9A199990476D1C7EE128
:10D9D0006002400F022809D003280DD004281898AF
:10D9E00001680DD00D60001D189070E11898EA17BD
:10D9F00001680D604A60F6E7189801680D80F2E74B
:10DA00000D70F0E718986A4601781172001D1890A1
:10DA10000020507202A80090012005E0189802C86A
:10DA2000189000200091C04361070DD5002101E04E
:10DA30000199491C0191B94212DA8142F8DB009A3E
:10DA4000515C0029F4D10BE0002101E00199491C4F
:10DA500001918142FADB019A0099895C0029F5D194
:10DA6000019904981A9B471A21463846199A00F0E2
:10DA700097FA0199401945180BE04FE02CE113E0AB
:10DA80004EE0009800990078491C00911A9A199963
:10DA900090470198401E0190401CF2D12146384623
:10DAA0001A9B199A10E137E00A2000210090019199
:10DAB0006002410F022907D0189A01CA1892C217B2
:10DAC0009446032908D00AE01898C01DC108C9006F
:10DAD00005C91891944607E000B2C217944604297C
:10DAE00002D140B2C1178C4600226146944506DA45
:10DAF0000A460021404291418C462D2102E0210539
:10DB000004D52B216A461173012103E0E10701D0FE
:10DB10002021F7E7029155E00A200AE0102008E0F2
:10DB2000102000900021042004430191082703E005
:10DB300008200021019100906002410F022907D0C6
:10DB4000189A01CA189200229446032908D008E0C6
:10DB50001898C01DC108C90005C91891944603E072
:10DB600080B2042900D1C0B200210291210729D539
:10DB70001199702906D0009A1021019B4A401A433E
:10DB800005D00EE040216A461173012108E061468C
:10DB9000014306D030216A46117311995173022155
:10DBA0000291009A0821019B4A401A430AD161461A
:10DBB000014301D1610705D530216A461173012166
:10DBC0007F1E02911199582904D035A10E910DA9FB
:10DBD0000D910DE037A1F9E76146019B009AF7F737
:10DBE0009DFA0E9B8C469B5C0D9A521E0D921370F3
:10DBF00061460143F0D10D9805A9081A2030019023
:10DC0000600703D501200004844300E00127019848
:10DC1000874201DD381A00E0002001990090411888
:10DC2000029809180498401A0490E00306D421468B
:10DC30001A9B199A049800F0B3F94519002706E0D9
:10DC400003A81A9AC05D199990476D1C7F1C029811
:10DC50008742F5DBE0030CD521461A9B199A0498FC
:10DC600000F09EF9451904E01A9A3020199990475E
:10DC70006D1C0099481E00900029F5DC08E00D9805
:10DC80000D990078491C0D911A9A199990476D1CAD
:10DC90000199481E01900029F1DC63E10928010087
:10DCA0003031323334353637383961626364656612
:10DCB00000000000303132333435363738394142D4
:10DCC000434445460000000000F05AF94519761C0F
:10DCD0003078002800D0E2E528461BB0F0BD600790
:10DCE00000D406271898C01DC108C90048680A68F2
:10DCF0000831C30FDB071891190001D09CA108E07F
:10DD0000210501D59BA104E0E10701D09AA100E023
:10DD10009AA1430011985B08109165280CD006DC8D
:10DD2000452809D046281DD0472841D141E0662822
:10DD300018D067283CD13CE00021112F01DB1120D5
:10DD400000E0781C0191009008A911A8FFF7E8FCF9
:10DD5000139905910021119A15927F1C1298019731
:10DD6000009150E00120C00703900120019008A914
:10DD7000009711A8FFF7D4FC139A1499059200227A
:10DD8000119B009212981593059A0192002901D0D7
:10DD9000104602E0791C40180190381A01D501980C
:10DDA00004E04042401E0090781C0190C01B02908D
:10DDB00043E0012F00DA01270021112F01DD11209E
:10DDC00000E038460191009008A911A8FFF7A8FCCF
:10DDD00013990591119A00211298159200910197BB
:10DDE00021070CD40599B94201DB019900E00191AA
:10DDF000012904DD159A491E515C302906D0B8422C
:10DE000001DA011D05DA0121029115E00199491E8F
:10DE1000EDE7002805DC0099411800910199091AE5
:10DE200003E0019A411C914200DD01910099401AE2
:10DE3000401C02900120C0070390200706D40299DD
:10DE40000198814202DB0020C04302900020694615
:10DE5000C87707AF012103980337C907884224D048
:10DE6000022011902B201290039800280CDA4042D7
:10DE700003902D20129007E00A210398F7F738F954
:10DE800030317F1E039039701199481E119000297E
:10DE9000F2DC03980028EFD1791E129808703078D0
:10DEA000202108404530BF1E387006A8C01BC01D89
:10DEB000039010980078002800D0012001994118A3
:10DEC0000298C0170918039809180498401A401EB0
:10DED0000490E00306D421461A9B199A049800F096
:10DEE0005FF8451910980078002803D01A9A1999FC
:10DEF00090476D1CE00324D521461A9B199A04987B
:10DF000000F04EF845191CE00098002807DB009946
:10DF10000598884203DD1598405C199901E019992C
:10DF200030201A9A904700986D1C401C009002986F
:10DF3000401E0290002804D11A9A2E201999904769
:10DF40006D1C0199481E01900029DDDC05E0387840
:10DF50001A9A7F1C199990476D1C0399481E0390CB
:10DF60000029F4DC21461A9B199A0498ACE60000BB
:10DF70002D0000002B000000200000000000000029
:10DF8000F8B5044600251E461746880404D405E06B
:10DF900039462020B0476D1C641EF9D52846F8BDCF
:10DFA000FFB50446002581B01E46C80301D53027C1
:10DFB00000E02027880404D505E038460399B047DF
:10DFC0006D1C641EF9D5284605B0F0BD4A68002ACC
:10DFD00006D00A68531C0B6010704868401E4860E9
:10DFE00070470000F8B54A002B4B520DD6182B4A4B
:10DFF0000C460546142E2BDA002E12DA284BF7F7C2
:10E00000F7F900221346F7F743FC40D2002C03DA5D
:10E010000124E40700253AE02046284337D0214C6C
:10E0200014E0214F0B46F7403B402B4331D01C4BB3
:10E03000F7F7DEF900221346F7F72AFC27D2002C67
:10E0400003DD01200005F0400419BC4300251EE05B
:10E05000332E1EDC33460027143BFF43DF4038429B
:10E0600017D00F4BF7F76EFA00221346F7F710FCA4
:10E070000DD2002C0ADD142E0CD03420811B01207F
:10E0800088404019A84200D2641C0546BD43214681
:10E090002846F8BD641CF9E701FCFFFF9C75008869
:10E0A0003CE4377E0000F03FFFFF0F007D2110B5FC
:10E0B000C900484300F001F810BD002140E000BF56
:10E0C00000BF00BF00BF00BF00BF00BF00BF00BF58
:10E0D00000BF00BF00BF00BF00BF00BF00BF00BF48
:10E0E00000BF00BF00BF00BF00BF00BF00BF00BF38
:10E0F00000BF00BF00BF00BF00BF00BF00BF00BF28
:10E1000000BF00BF00BF00BF00BF00BF00BF00BF17
:10E1100000BF00BF00BF00BF00BF00BF00BF00BF07
:10E1200000BF00BF00BF00BF00BF00BF00BF00BFF7
:10E1300000BF00BF00BF00BF00BF00BF00BF491C41
:10E140008142BCD370470000FEB50446002006465D
:10E1500001906079764940000F5A617875482578BA
:10E16000491E6A4601631170042D7CD0072D7AD0B8
:10E1700000210291217801736E49E3790122920511
:10E180008969002B71D0914381616A48217A41737A
:10E19000217A82698907890B0A4382610021042060
:10E1A00000F04DFB3A4664492E2000F03DFB6846E6
:10E1B0000078FFF701FA614F0522785D8100401871
:10E1C0005F49431807212B2000F048FB5D49029866
:10E1D00001220B180B21282000F040FB785D5A49E2
:10E1E00080000A580C21282000F029FBE0795749CB
:10E1F00080004018A1794900425A0221272000F0EE
:10E2000013FB68460078524940000A5A042127202F
:10E2100000F00AFBE07900282BD0A07804282ED04B
:10E2200028206946087220220621272000F0FCFAE7
:10E2300002AB01222621272000F010FB684600785F
:10E24000444900014018E1788900425808212720FC
:10E2500000F0F5FAA17A601C627A0902114313D02A
:10E2600016E000E001E0012183E71143FF0881612E
:10E270008BE764220621272000F0D6FADEE7102083
:10E28000694608720246CFE733490172090A4172B2
:10E29000417A007A0A0202432021272000F0C4FAC2
:10E2A0002E4F0C2123203A6800F0C9FA6846007806
:10E2B00004214000C0198288232000F0B5FAA0791B
:10E2C00000280AD0E07926490122431800212120A4
:10E2D00000F0C4FA0320012601902A07120F100152
:10E2E0000243607800218007000B0243019800057B
:10E2F0000243700402432079C0064009024360795A
:10E30000C00602431F2000F09AFAA078617801232A
:10E31000084302040748DB030261E179490319431A
:10E320000A4302610021082000F089FA0020FEBDA6
:10E3300028EE0008102E002004280000D0ED000870
:10E34000C4010020E2010020D8ED0008F8ED00082B
:10E3500004EE000808EE000841100000F0ED00088F
:10E36000E401002038B50C4607498A8B002102439E
:10E370002C2000F059FA684604706B4601220621F1
:10E380002C2000F06BFA38BD102E002010B5FFF7DE
:10E3900000F910BD10B504460421362000F0FCF849
:10E3A0000121C902002C01D0084300E08843024645
:10E3B0000421362000F043FA10BD000038B540209B
:10E3C0006946087000210E2000F0E6F8044600229D
:10E3D00011460E2000F033FA6B46012200210D2079
:10E3E00000F03CFA074A00210F2000F028FA00F064
:10E3F00001FA224600210E2000F021FA02480021F5
:10E40000017338BDF8FF2724302E0020FEB50546E5
:10E41000042069460870514C002060752146203167
:10E42000206348710873A0836063A06300F0E2F882
:10E430004B4E206002E000F0DDF82060B042FAD1DF
:10E440000020FFF7D7F800F0D5F8464E206030786E
:10E45000242801D9243806E00621F6F749FE0622D1
:10E46000101A40010843020601040A4301020A434C
:10E470000243B260706000211E2000F0E0F900F05D
:10E48000B9F820606B4601220021242000F0E6F953
:10E490001E20FFF723F986B2300AA0730420FFF78D
:10E4A0001DF9074600F0A6F820603806000E0DD0D2
:10E4B00002206946087101AB012212212D2000F0D3
:10E4C000CDF9A08B012109030843A08300F092F845
:10E4D00020600620FFF702F960600720FFF7FEF8D2
:10E4E000A060F006C00E207501D110202075C0B2CA
:10E4F00000F0F0F9E80707D0FFF7D7F8A08B01216B
:10E50000C9020843A0830AE00521362000F02EF856
:10E510001549084002460521362000F085F9012002
:10E52000FFF768F80021042000F036F8A061002110
:10E53000262000F031F81521890308430246002106
:10E54000262000F07CF900222621362000F06CF90C
:10E5500000F050F820600020FEBD0000102E0020CA
:10E560003001CADEB8010020FFFD000038B5094CBB
:10E5700089B280B26B46022200F042F8002806D130
:10E5800068464078010268460078081884B2204640
:10E5900038BD0000FFFF000038B50024E44389B215
:10E5A00080B26B46042200F02BF8002806D103212C
:10E5B0006846435C2202D418491EFAD5204638BD6D
:10E5C00038B500246B4603222821272000F018F8D4
:10E5D000022069460B5C2202D418401EFAD5E002E4
:10E5E00002D50348204338BDE002C00A38BD000010
:10E5F0000000F0FF10B500210846FFF7CDFF10BD69
:10E6000038B5002909D0402420436C462070C8B298
:10E610007F2906D8607002200AE069460870012050
:10E6200006E0802420436C466070C809A070032077
:10E63000694600F019FB38BD10B5144603460A467A
:10E6400021461120FFF7DCFF10BD10B5034605225F
:10E6500000211520FFF7D4FF10BD10B50346052299
:10E6600000211720FFF7CCFF10BD38B5054600206C
:10E670006946087000F0BEF8FF2401342246002DE0
:10E6800001D00322120200210D2000F0CDF8002D50
:10E6900013D06B46012203210F20FFF7B1FF68461C
:10E6A0000078000709D5FFF789FE224600210D20DA
:10E6B00000F0BAF80020C04338BD002038BD10B5C6
:10E6C000044600211A20FFF767FF000D2203000512
:10E6D000120B024300211A2000F0B1F810BD000017
:10E6E00010B5024602492E2000F09EF810BD000031
:10E6F00004180000F8B505466B46012203210420EA
:10E70000FFF77EFF0126114C3607002D0DD02A465B
:10E7100000210C2000F088F8694608781021084391
:10E7200069460870A069304307E069460878EF2120
:10E73000084069460870A069B0430B46A0610122F9
:10E740000321042000F08AF8F8BD0000102E0020FC
:10E7500010B502460021182000F066F810BD000038
:10E76000F8B50746002568460570B807204C2E46C8
:10E7700000280ADA8020694608706B4601220021D1
:10E780000D2000F06BF801202073F8076946087827
:10E7900021D006210843694608706B4601220021FA
:10E7A0000D2000F05BF803210F20FFF7DFFE812131
:10E7B000C900084219D04020694608706B46012202
:10E7C00000210D2000F04AF80020FFF7E3FD0025AE
:10E7D0002673ED4309E002210843694608706B4641
:10E7E000012200210D2000F039F82846F8BD000074
:10E7F000302E00201CB56B46012203210F20FFF7AD
:10E80000FFFE684600784022C1091040C90140005F
:10E81000814208D0012069460871024601AB0321FC
:10E820000D2000F01BF81CBD08B56B461A70120ACB
:10E830005A7089B280B2022200F010F808BD38B5D3
:10E8400000236C46E254120A5B1C042BFADB89B2EB
:10E8500080B22346042200F001F838BD38B5802488
:10E86000002909D0C02528436D462870C8B27F29E9
:10E8700007D86870022009E020436946087001202B
:10E8800004E020436870C809A8700320694600F0BE
:10E8900035FA38BD10B51446012312189B029A426E
:10E8A00002D90020C04310BD0B46821E214609201C
:10E8B000FFF7D4FF002010BD10B5054A8905126985
:10E8C00001430A4300210820FFF7B9FF002010BDD3
:10E8D000102E002038B504466B4601220E212B2055
:10E8E000FFF78EFE68460078E10640094001C90E38
:10E8F0000143684601706B4601220E212B20FFF771
:10E90000ADFF38BD7CB5002425466846FFF79DFE67
:10E9100004206946220E2D02154322020C5C14438A
:10E92000401EF7D5204629467CBD7CB500242546EF
:10E930006846FFF792FE04206946220E2D02154319
:10E9400022020C5C1443401EF7D5204629467CBDAC
:10E95000F8F7B8FFFDF78EFBFBF770FFFBF736FF0C
:10E96000FCF70EF8FCF79EF8FCF7B8F8FCF724F873
:10E97000FCF748F82348224901600021416081608A
:10E980000162214A416242618162F9F763F800281D
:10E9900001D072B6FEE7FCF757FCF7F743FFF7F735
:10E9A00011FFFF2007214130FFF7DCFCFFF7EEFCF1
:10E9B000F7F72AFBF7F738FAFDF742F8FCF76AFB9E
:10E9C000FF20000203461A461146FDF71DF8FF24FA
:10E9D000F5342046F8F75AFDFF20000403461A4696
:10E9E0001146FDF711F82046F8F750FDF7F744FA05
:10E9F000FEF7DEFCF7F7C2FBFDF7B8FCF6E7000018
:10EA0000007C004004050020FFFF000010B5044614
:10EA1000FBF7CAFA4E20FBF799FAFBF701FBE0B2CD
:10EA2000FBF794FAFBF7FCFAFBF7BEFA4F20FBF773
:10EA30008DFAFBF7F5FA0020FBF75AFA0446FBF7CC
:10EA4000CFFA204610BD70B50D460446FBF7ACFA70
:10EA50004E20FBF77BFAFBF7E3FAE0B2FBF776FA1E
:10EA6000FBF7DEFA2846FBF771FAFBF7D9FAFBF75A
:10EA7000B7FA0A20FFF721FB70BD000010B5242172
:10EA8000002000F04DF81B48FFF717FB00210F2076
:10EA900000F046F80521102000F042F80421112072
:10EAA00000F03EF883217F2000F03AF869217F20B2
:10EAB00000F036F8BD217F2000F032F80E480078D3
:10EAC000262804D1002240218C2000F019F80120D2
:10EAD00000F02AF8094814210187282000F020F8C6
:10EAE0000A20FFF7EAFA012000F036F8012000F0D2
:10EAF00043F810BD204E0000A00100206407002054
:10EB0000F8B517460E4605460024FFF77FFF394645
:10EB1000B44331402143284600F002F80020F8BDFC
:10EB200010B5FFF790FF10BD10B500280AD00021E6
:10EB30002720FFF7F5FF04211920FFF7F1FF8721B8
:10EB4000162005E000211620FFF7EAFF002119201A
:10EB5000FFF7E6FF10BD000010B5002801D000222D
:10EB600000E0802280211120FFF7CAFF0148FFF753
:10EB7000A4FA10BDA086010010B5002811D0012113
:10EB80002F20FFF7CDFF62213020FFF7C9FF46217C
:10EB90003120FFF7C5FF32210846FFF7C1FFA22150
:10EBA00000E022213320FFF7BBFF10BD0C480D4AC7
:10EBB0000188914210D1C18832290DD3C18E4329D9
:10EBC0000AD8818F012907D8C08F012804D80448AA
:10EBD00040308088012801D901207047002070470B
:10EBE00064070020AA55000010B50124A4022146A4
:10EBF0001948F6F7DCFA224617491848F7F76CFE71
:10EC00001548174902888A4224D00180154981801D
:10EC10007D21C900C1800A210181002141818181BA
:10EC20000122C28181834323C386022303874B1EB3
:10EC300043878287C287024640321184518491847F
:10EC4000C183918014238382E12011820001D0844A
:10EC500000F032F810BD00006407002000FC00083E
:10EC6000AA55000034120000F0B58C460025FF269E
:10EC70000F4901368E620F4C08E067467F5DE76002
:10EC8000A768FF07FCD0E7681F706D1C8542F4DBA6
:10EC90000020074606E0E760A568ED07FCD0E568C0
:10ECA0001D54401C9042F6D38E610020F0BD000040
:10ECB000000400500030014070B5FFF777FF0028D6
:10ECC00001D0012070BD72B60124074DA402214677
:10ECD0002846F7F7E7FD002804D0224603492846D6
:10ECE000F7F786FE62B670BD00FC000864070020DE
:10ECF000002100E0491C8142FCD37047F0B500259B
:10ED0000FF260F4F9C4601360B46BE620D4C06E0B7
:10ED1000595DE160A168C907FCD0E1686D1C8542BE
:10ED2000F6DB002007E06146095CE160A168C907E5
:10ED3000FCD0E168401C9042F5D3BE610020F0BDDC
:10ED400000040050003001409CEF000803C00008A0
:10ED500084EF000849BD00085CEF000835BC0008DE
:10ED600040EF000871BB000814EF000819BB000851
:10ED700074EF0008E9BC00087CEF0008EDBC000857
:10ED800000EF000855BD00086CEF0008F9BE000850
:10ED900008EF000851BE000834EF000879BF0008F2
:10EDA0008CEF0008F1BD000854EF0008FDBB00081F
:10EDB0002CEF0008C5BB00084CEF0008E1BA0008C2
:10EDC00020EF0008A9BA000864EF0008F9BF0008A6
:10EDD0000000010203040005405C0000A05C040088
:10EDE000C06C0800805C0400E03F1E00E07D1E0057
:10EDF00007A9022570889B880A00160001000600FA
:10EE00000100020087008D002D001A3152001A33D4
:10EE10009A001A351D011A376B003B31BE003B3397
:10EE20005E013B3596023B37000099599959EB51E9
:10EE30008F421E45142E0080EB51F5283333E13A02
:10EE4000703DE13AC235852BC2353333C235C23508
:10EE5000AE47E13A5138A3305138000000000000BD
:10EE600000000102030406070809030406080C1049
:10EE70001820300000000001020304004040404020
:10EE8000404040404041414141414040404040407D
:10EE90004040404040404040404040400502020267
:10EEA00002020202020202020202020220202020CA
:10EEB00020202020202002020202020202909090D4
:10EEC00090909010101010101010101010101010C2
:10EED000101010101010100202020202028888881E
:10EEE0008888880808080808080808080808080822
:10EEF0000808080808080802020202407CEE000820
:10EF00007365745F616463007365745F6465765FE5
:10EF10006964000064656275675F6F666600000083
:10EF2000626565705F6F6666000000006770735F02
:10EF30006F6666007365745F77696669000000003C
:10EF400064656275675F6F6E0000000062656570E2
:10EF50005F6F6E006770735F6F6E0000696E666F43
:10EF600000000000736C6565700000007365745FDD
:10EF7000697000007274635F676574007274635F28
:10EF8000736574007265626F6F7400007365745FFF
:10EF9000636F6E7472617374000000007465737443
:10EFA000000000002B2B2B0D0000000061742B6A69
:10EFB0006F696E3D6F7461612C31300D000000008F
:10EFC00061742B63683D636E3437302C330D000061
:10EFD00061742B64723D350D0000000061742B617B
:10EFE00070706575693D3532363937333639366577
:10EFF0003637343834360D0061742B636C617373AB
:10F000003D610D0061742B6170706B65793D3262FA
:10F010003765313531363238616564326136616267
:10F0200066373135383830396366346633630D00FE
:10F0300061742B6D6F64653D6D61630D00000000B0
:10F0400061742B6164723D6F66660D0061742B7292
:10F0500065626F6F740D000061742B736C65657071
:10F060003D6C696768742C302C6C6576656C2C6C13
:10F070006F770D0061742B6465766575693D343773
:10F0800033363534396630303331253034780D003D
:10F09000636C6561720000006C730000BCF00008D6
:10F0A00000000020A8040000385C000848F10008B7
:10F0B000A8040020C030000084D50008014D1204CF
:10F0C00012500236801405021415090901026281EA
:10F0D000029101072452030CE5800CC9BC7A0C0F85
:10F0E00013A4EF140830F01B08AC081AF8041A74C3
:10F0F0000C1ADC081A04081AD0081AC0041A400CAA
:10F100001A58041A4C0441022327130704380D0926
:10F110001E080540082609104008560A131D043B26
:10F1200008BE053ED8BC401008949204022120324B
:10F13000021A90841341971B0898081AF50801FFDA
:08F1400001FF017672010000DD
:04000005080050C1DE
:00000001FF
